:0200000480007A
:10000000B72F0000938F0F8073900F306F00400365
:100010001300000013000000130000001300000094
:100020001300000013000000130000001300000084
:100030001300000013000000130000001300000074
:100040009702000093824211739052309300000097
:10005000130100009301000013020000930200004E
:100060001303000093030000130400009304000036
:10007000130500009305000013060000930600001E
:100080001307000093070000130800009308000006
:100090001309000093090000130A0000930A0000EE
:1000A000130B0000930B0000130C0000930C0000D6
:1000B000130D0000930D0000130E0000930E0000BE
:1000C000130F0000930F0000971102009381C1D617
:1000D000170502001305055B97A50300938545846A
:1000E00013060000EF00001A170502001305454E25
:1000F000970502009385055413060000EF00801851
:1001000017B503001305058297C503009385458144
:1001100037B6ABAB1306B6BAEF00C01617C1030073
:1001200013014180EFA0000D9392120093D21200B0
:100130009382D2FF638A02008322010013014100EF
:100140006F0000177300203083220100130141006B
:10015000730020301301C1FF23205100F32220340B
:10016000E3C402FC8322010013014100130141F8A2
:1001700023221100232421002326310023284100BB
:10018000232A5100232C6100232E71002320810299
:10019000232291022324A1022326B1022328C10293
:1001A000232AD102232CE102232EF1022320010570
:1001B0002322110523242105232631052328410567
:1001C000232A5105232C6105232E71052320810745
:1001D000232291072324A1072326B1072328C1073F
:1001E000232AD107232CE107232EF107732520347E
:1001F000F3251034130601006F000000731015344E
:1002000083204100032181008321C10003220101D9
:1002100083224101032381018323C10103240102BD
:1002200083244102032581028325C10203260103A1
:1002300083264103032781038327C1030328010485
:1002400083284104032981048329C104032A010569
:10025000832A4105032B8105832BC105032C01064D
:10026000832C4106032D8106832DC106032E010731
:10027000832E4107032F8107832FC1071301C10775
:10028000730020302320C5006376B50013054500B8
:100290006FF05FFF678000000000000000000000BA
:1002A000000000000000000000000000000000004E
:1002B000130101F8232011002322210023243100FF
:1002C0002326410023285100232A6100232C71009A
:1002D000232E8100232091022322A1022324B10294
:1002E0002326C1022328D102232AE102232CF10272
:1002F000232E010323201105232221052324310568
:100300002326410523285105232A6105232C710545
:10031000232E8105232091072322A1072324B1073F
:100320002326C1072328D107232AE107232CF1071D
:100330009702020083A2022D23A02200F322103490
:10034000232E5106EF00C03B170102000321812B31
:10035000032101008322C10773901234B7220000E9
:100360009382028873A00230832001000322C1001F
:100370008322010103234101832381010324C1015D
:100380008324010203254102832581020326C10241
:100390008326010303274103832781030328C10325
:1003A000832801040329410483298104032AC10409
:1003B000832A0105032B4105832B8105032CC105ED
:1003C000832C0106032D4106832D8106032EC106D1
:1003D000832E0107032F4107832F81071301010893
:1003E00073002030970202009382C22923A01200DA
:1003F00023A2220023A4320023A6420023A85200F5
:1004000023AA620023AC720023AE820023A09202D2
:1004100023A2A20223A4B20223A6C20223A8D202CC
:1004200023AAE20223ACF20223AE020323A01205A8
:1004300023A2220523A4320523A6420523A85205A0
:1004400023AA620523AC720523AE820523A092077E
:1004500023A2A20723A4B20723A6C20723A8D20778
:1004600023AAE20723ACF207EF601029170102006C
:1004700003214119032101008322C1077390123423
:10048000B72200009382028873A00230832001000B
:100490000322C1008322010103234101832381013F
:1004A0000324C10183240102032541028325810223
:1004B0000326C10283260103032741038327810307
:1004C0000328C103832801040329410483298104EB
:1004D000032AC104832A0105032B4105832B8105CF
:1004E000032CC105832C0106032D4106832D8106B3
:1004F000032EC106832E0107032F4107832F810797
:1005000013010108730020309702020093828217C2
:1005100083A0020003A1420083A1820003A2C200C3
:1005200083A2020103A3420183A3820103A4C201A7
:1005300083A4020203A5420283A5820203A6C2028B
:1005400083A6020303A7420383A7820303A8C2036F
:1005500083A8020403A9420483A9820403AAC20453
:1005600083AA020503AB420583AB820503ACC20537
:1005700083AC020603AD420683AD820603AEC2061B
:1005800083AE020703AFC20983AF82076780000012
:1005900073700430130101F823201100232221007D
:1005A000232431002326410023285100232A6100FF
:1005B000232C7100232E8100232091022322A102EB
:1005C0002324B1022326C1022328D102232AE102D7
:1005D000232CF102232E01032320110523222105C0
:1005E000232431052326410523285105232A6105AB
:1005F000232C7105232E8105232091072322A10797
:100600002324B1072326C1072328D107232AE10782
:10061000232CF1079702020083A2C2FE23A022002E
:10062000232E1106EF30802917010200032181FDDE
:10063000032101008322C10773901234B722000006
:100640009382028873A00230832001000322C1003C
:100650008322010103234101832381010324C1017A
:100660008324010203254102832581020326C1025E
:100670008326010303274103832781030328C10342
:10068000832801040329410483298104032AC10426
:10069000832A0105032B4105832B8105032CC1050A
:1006A000832C0106032D4106832D8106032EC106EE
:1006B000832E0107032F4107832F810713010108B0
:1006C00073002030737004306F00000073104530E9
:1006D000678000007325403073F04330678000006E
:1006E00097070000938747FE232EB5FE2322C5FA05
:1006F000232635F82320F5F8130505F86780000058
:10070000130101FF23261100EF60C07BEF20C051D1
:10071000631805008320C1001301010167800000F8
:100720008320C100130101016F3040199307850038
:100730001307F0FF2322F5002324E5002326F5000C
:100740002328F500232005006780000023280500EA
:10075000678000008327450023A2F50003A78700D8
:1007600023A4E50003A787002322B70023A4B70032
:1007700023A8A50083270500938717002320F500F1
:100780006780000003A605009307F0FF13078500AC
:100790006316F6006F008003138707008327470066
:1007A00083A60700E37AD6FE23A2F50023A4B700B0
:1007B00023A4E5002322B70023A8A5008327050072
:1007C000938717002320F5006780000003270501A9
:1007D000832747006FF05FFD0327450083268500D0
:1007E000832705012324D70003278500832645009E
:1007F0002322D70003A747006316A700032785001D
:1008000023A2E7002328050003A507001305F5FF31
:1008100023A0A70067800000032605049387050036
:10082000630406028325C50003274500B385C50080
:100830002326B50063E6E500832505002326B500E1
:10084000138507006F50404467800000130101FFCB
:100850002324810023261100130405002322910084
:10086000EF30103A83278404635AF004832744024C
:1008700063860704930444026F0000028327840404
:100880009387F7FF2324F404832784046358F0023A
:10089000832744026384070213850400EF30406518
:1008A000E30E05FCEF301012832784049387F7FFD3
:1008B0002324F40483278404E34CF0FC9307F0FF23
:1008C0002324F404EF301037EF30903383274404AF
:1008D000635AF00483270401638607049304040128
:1008E0006F000002832744049387F7FF2322F40458
:1008F000832744046358F0028327040163840702BA
:1009000013850400EF30C05EE30E05FCEF30900B62
:10091000832744049387F7FF2322F40483274404A6
:10092000E34CF0FC9307F0FF2322F404032481003E
:100930008320C10083244100130101016F30902FF7
:10094000630A0508130101FE232C8100130405002E
:10095000232E1100232A910023282101232631016F
:1009600013890500EF30D029832404048325C403B0
:100970008329040013850400EF90405D1307F0FF06
:10098000232C0402B3079540B387F9003385A900EF
:100990002322E4042322A400232434012326F40088
:1009A0002324E404631C09028327040163920704DF
:1009B000EF3050288320C1010324810183244101A9
:1009C000032901018329C10013051000130101024D
:1009D00067800000737004306F000000130504018D
:1009E000EFF0DFD413054402EFF05FD46FF05FFC4B
:1009F00013050401EF30C04F93071000E31AF5FA16
:100A0000EFF01FB96FF0DFFA631605007370043062
:100A10006F000000130101FE232A91002328210109
:100A200023263101232E1100232C8100930405007D
:100A300013890500930906006380050AEF900051B1
:100A400013055505EF50C00313040500630E050898
:100A5000930745052320F500232E94022320240527
:100A6000EF30101A832404048325C40303290400EF
:100A700013850400EF90804D9306F0FF232C0402B1
:100A8000B30795403307A900B307F9002322D40424
:100A90002322E4002326F4002324D40413050401B4
:100AA00023242401EFF09FC813054402EFF01FC870
:100AB000EF30501823083405130504008320C101CA
:100AC0000324810183244101032901018329C100F9
:100AD000130101026780000013054005EF40507AC2
:100AE0001304050063160500737004306F000000E6
:100AF000232084006FF05FF66316050073700430E6
:100B00006F0000006376B500737004306F00000062
:100B1000130101FF23248100130620001384050024
:100B20009305000023261100EFF01FEE630C050073
:100B3000232C85028320C1000324810013010101BD
:100B400067800000737004306F000000130101FB28
:100B50002326110423248104232291042320210528
:100B6000232E3103232C4103232A5103232861031D
:100B7000232671032326C10063060528638C0526FE
:100B800093072000639CF6000327C503930710001A
:100B90006306F700737004306F00000013890600CD
:100BA0009384050013040500EF30C065631A050047
:100BB0008327C10063860700737004306F00000054
:100BC000EF301004032784038327C403130B0000B2
:100BD000930B20009309F0FF130A0401930A4402C7
:100BE0006364F710630479238327C10063820736A7
:100BF00063160B0013058101EF30404AEF3090037C
:100C0000EF109074EF30C07F832744046394370162
:100C100023220404832784046394370123240404D7
:100C2000EF3050019305C10013058101EF30004AF8
:100C300063160530EF30C07C032784038327C40389
:100C40006304F710EF30007FEF30807B832784044C
:100C50006346F0026F00000313850A00EF3040295D
:100C600063040500EF300056832784049387F7FF61
:100C70002324F404832784046356F000832744026A
:100C8000E39C07FC23243405EF30C07AEF30407733
:100C9000832744046346F0026F00000313050A0033
:100CA000EF30002563040500EF30C0518327440472
:100CB0009387F7FF2322F404832744046356F0004C
:100CC00083270401E39C07FC23223405EF30807660
:100CD000EF20001B130B1000EF30807203278403FA
:100CE0008327C403E370F7F00326040463040612A9
:100CF000631A091E0325840093850400EF40D07811
:100D0000832784008326040403274400B387D70085
:100D10002324F40063E4E71083278403832604007C
:100D200003274402938717002324D400232CF402C2
:100D30006300071013054402EF30801B9307100077
:100D40006318F50E6F004014EF30C06E8325C100AC
:100D500013050A00EF20D06CEF30806A83278404EB
:100D60006346F0026F00000313850A00EF3040185D
:100D700063040500EF300045832784049387F7FF61
:100D80002324F404832784046356F0008327440259
:100D9000E39C07FC23243405EF30C069EF30406644
:100DA000832744046346F0026F00000313050A0022
:100DB000EF30001463040500EF30C0408327440483
:100DC0009387F7FF2322F404832744046356F0003B
:100DD00083270401E39C07FC23223405EF30806560
:100DE000EF20000AE31805EEEFF08FFA130B100066
:100DF0006FF09FEE83270504E38407D873700430F7
:100E00006F000000737004306F00000003260404BC
:100E1000631006088327040063860704832784037E
:100E20000327440293871700232CF402E31407F0EE
:100E3000EF304060130510008320C10403248104B7
:100E400083244104032901048329C103032A810364
:100E5000832A4103032B0103832BC10213010105E4
:100E60006780000003254400EF30804C8327840313
:100E7000032744022322040093871700232CF40243
:100E8000E31A07EAE30605FAEFF08FF06FF05FFA76
:100E90000325C40093850400EF40105F83270404FA
:100EA0000327C40083260400B307F0403307F7008C
:100EB0002326E400637ED70403274400B307F7002A
:100EC0002326F40013072000832744026304E90467
:100ED0000327840313071700232CE402E38A07F493
:100EE0006FF05FE50325C40093850400EF40D059FF
:100EF000832704040327C40083260400B307F040BB
:100F00003307F7002326E400E37ED7FA6FF0DFFA19
:100F10008327440203278403E30C07FA032784038F
:100F20001307F7FF232CE40203278403130717009A
:100F3000232CE402E38E07EE6FF0DFDF13050400DD
:100F4000EFF0DF90EF10D073130500006FF0DFEECD
:100F5000EF30404E130500006FF01FEE130101FF4C
:100F600023229100930405001305400523248100EA
:100F700023261100EF40D03013040500630C050454
:100F8000232C05029307F0FF2322F504130710001A
:100F900013050501232EE4022324F4042322040074
:100FA0002320040023240400232604002320040417
:100FB00023089404EFF08FF713054402EFF00FF7C6
:100FC00093060000130600009305000013050400BB
:100FD000EFF0DFB7130504008320C1000324810074
:100FE00083244100130101016780000063040504AC
:100FF000130101FF232481002322910023261100E5
:10100000232021010329450013040500EF30801E31
:10101000930400006304A9028320C100032481001B
:1010200013850400032901008324410013010101F9
:1010300067800000737004306F0000008327C400D5
:10104000930410009387F7FF2326F400E39607FC30
:10105000930600001306000093050000130504002A
:10106000EFF0DFAE6FF05FFB6302050A63880508EF
:10107000130101FE232C8100232A91002328210142
:1010800023244101232E1100232631019307200040
:101090009384060013090600138A05001304050053
:1010A000639CF6000327C503930710006302F70A49
:1010B000737004306F000000EFF0CFE1032784036A
:1010C0008327C403930905006366F70493040000B3
:1010D00013850900EFF08FDF8320C1010324810114
:1010E0001385040003290101832441018329C100E0
:1010F000032A810013010102678000008327050491
:10110000E38807F6737004306F00000073700430DA
:101110006F00000003260404631E060C83270400EE
:1011200063860712832784031307F0FF9387170052
:10113000232CF402832784046388E70E8327840426
:1011400093041000938717002324F4046FF05FF8D2
:10115000EFF04FD8032784038327C40393090500C6
:101160006360F70603260404E30A06FA0325C400B5
:1011700093050A00EF405031832704040327C4007D
:1011800083260400B307F0403307F7002326E4006A
:101190006378D70003274400B307F7002326F40041
:1011A00093072000E390F4F883278403E38C07F689
:1011B000832784039387F7FF232CF4026FF09FF6B5
:1011C00003260404E30C06F40325C40093050A0077
:1011D000EF40902B832704040327C40083260400D8
:1011E000B307F0403307F7002326E400E364D7FA9F
:1011F0006FF09FFBE39C04F60325840093050A002F
:10120000EF409028832784008326040403274400AA
:10121000B387D7002324F400E3E6E7F08327040034
:101220002324F4006FF01FF083274402930410007E
:10123000E38007EA13054402EF20904BE30A05E838
:10124000E30809E8232099006FF09FE80325440094
:10125000EF30000E232204006FF0DFEC6302050A7A
:101260008327050463860700737004306F00000055
:1012700083270500638A0708130101FE232C8100E0
:10128000232A91001304050023282101232631017C
:10129000232E110013890500EFF0CFC30327840329
:1012A0008327C40393090500930400006376F702C3
:1012B000832784031307F0FF93871700232CF4027E
:1012C00083278404638AE70483278404930410003B
:1012D000938717002324F40413850900EFF00FBF50
:1012E0008320C10103248101138504000329010126
:1012F000832441018329C10013010102678000009A
:10130000737004306F00000083274500E38607F602
:10131000737004306F000000832744026396070057
:10132000930410006FF05FFB13054402EF20503C64
:10133000E30805FEE30609FE930710002320F900E9
:101340006FF01FFE130101FC232E1102232C8102DA
:10135000232A910223282103232631032324410336
:10136000232251032326C10063060528638C05262A
:10137000938A06009389050013040500EF20906806
:10138000631A05008327C100638607007370043069
:101390006F000000EF30C006832784036394071CAE
:1013A0008327C1006380071013058101EF20104FD0
:1013B0009304F0FF13094402130A0401EF3080077D
:1013C000EF108078EF30C0038327440463949700C4
:1013D00023220404832784046394970023240404B1
:1013E000EF3040059305C10013058101EF20104E39
:1013F00063100524EF30C00083278403638A070A43
:10140000EF304003EF20D07F832784046346F0024F
:101410006F00000313050900EF20902D6304050001
:10142000EF20505A832784049387F7FF2324F40482
:10143000832784046356F00083274402E39C07FC5F
:1014400023249404EF20107FEF20907B8327440413
:101450006346F0026F00000313050A00EF205029D5
:1014600063040500EF201056832744049387F7FF99
:101470002322F404832744046356F00083270401E5
:10148000E39C07FC23229404EF20D07AEF10501F36
:10149000EF201077832784036396070C8327C1000E
:1014A000E39E07F0EF201079130500006F00800F16
:1014B000EF20507883270400638807108325C1003C
:1014C00013050900EF20C075EF2090738327840473
:1014D0006346F0026F00000313050900EF2050215E
:1014E00063040500EF20104E832784049387F7FFE1
:1014F0002324F404832784046356F00083274402E2
:10150000E39C07FC23249404EF20D072EF20506F5B
:10151000832744046346F0026F00000313050A00AA
:10152000EF20101D63040500EF20D04983274404F9
:101530009387F7FF2322F404832744046356F000C3
:1015400083270401E39C07FC23229404EF20906E80
:10155000EF10101363040508EF20906A83278403BB
:10156000E38E07F293850900130504008324C40069
:10157000EFF08FAA63940A088327840303270400EB
:101580009387F7FF232CF40263160700EF20D07136
:101590002322A4008327040163920708EF209069A7
:1015A000130510008320C103032481038324410316
:1015B000032901038329C102032A8102832A4102EC
:1015C0001301010467800000EF20906303254400AD
:1015D000EF201046EF2010666FF05FEEEFE05FFB4C
:1015E0006FF09FF783270504E38407D873700430F6
:1015F0006F000000737004306F0000008327440206
:1016000023269400E38C07F813054402EF20500EC4
:10161000E30605F8EFE0DFF76FF05FF8130504016C
:10162000EF20100D93071000E31AF5F66FF09FFE00
:1016300013050400EFF08FA1EF10900413050000D4
:101640006FF05FF663000506130101FF232481009C
:101650002320210123261100232291008324450009
:101660001389050013040500EF20D0386380A4041B
:1016700093060000130609009305000013050400FB
:10168000EFF05FCC93071000630CF5028320C100DC
:101690000324810083244100032901001301010177
:1016A00067800000737004306F0000008327C4005F
:1016B00013051000938717002326F4006FF01FFD19
:1016C0008327C400938717002326F4006FF01FFCC4
:1016D000630805066386050C130101FE232C8100B7
:1016E000232A9100232821012326310123244101AB
:1016F00013040500232E1100130906009389050029
:10170000EFE05FFD83278403130A050093040000C4
:10171000639C070213050A00EFE05FFB8320C10111
:10172000032481011385040003290101832441015D
:101730008329C100032A8100130101026780000090
:10174000737004306F000000032604046304060273
:101750008325C40083274400B385C5002326B40035
:1017600063E6F500832504002326B40013850900F1
:10177000EF408051832784031307F0FF9387F7FF1F
:10178000232CF402832744046384E7028327440460
:1017900093041000938717002322F4046FF09FF73F
:1017A00083270504E38A07F2737004306F0000009A
:1017B0008327040163960700930410006FF09FF5E0
:1017C00013050401EF20C072E30805FEE30609FEDD
:1017D000930710002320F9006FF01FFE6306050831
:1017E00083270504638A050863840708130101FE43
:1017F000232C8100232A9100232821012324410145
:1018000013040500232E110023263101138A05003D
:10181000EFE05FEC832784031309050093040000C5
:10182000638E07008329C40093050A001305040092
:10183000EFE09FFE930410002326340113050900F6
:10184000EFE0DFE88320C101032481011385040058
:1018500003290101832441018329C100032A810056
:101860001301010267800000737004306F000000F4
:10187000737004306F000000E38C07FE7370043057
:101880006F00000063160500737004306F000000E5
:10189000130101FF232481001304050023261100F6
:1018A000EF20103603248403EF20D0388320C100BA
:1018B0001305040003248100130101016780000067
:1018C00063160500737004306F000000130101FF00
:1018D000232611002324810013040500EF20503239
:1018E000832784030324C4033304F440EF2090349B
:1018F000130504008320C1000324810013010101AA
:1019000067800000630605000325850367800000EB
:10191000737004306F0000006308050497870300AC
:10192000938747FC03A747006304E50403A7C700A8
:101930006302E50803A74701630AE50603A7C70199
:101940006302E50603A74702630AE50403A7C7028B
:101950006302E50403A74703630AE50203A7C7037D
:101960006302E5026F40C029737004306F0000000D
:101970001307000013173700B387E70023A0070001
:101980006F400028130770006FF0DFFE1307600040
:101990006FF05FFE130750006FF0DFFD130740008C
:1019A0006FF05FFD130730006FF0DFFC13072000BE
:1019B0006FF05FFC130710006FF0DFFB0325C50419
:1019C000678000002326B5046780000003450505F5
:1019D00067800000630805000325850313351500A3
:1019E00067800000737004306F000000630C050016
:1019F000832785030325C5033305F54013351500FB
:101A000067800000737004306F0000009787030048
:101A1000938747ED03A707006300070403A7870028
:101A20006308070403A707016308070403A78701E6
:101A30006308070403A707026308070403A78702D4
:101A40006308070403A70703630C070403A78703BE
:101A500063040704678000001307000013173700B2
:101A6000B387E70023A0B70023A2A7006780000088
:101A7000130710006FF09FFE130720006FF01FFE8A
:101A8000130730006FF09FFD130740006FF01FFD3C
:101A9000130750006FF09FFC130770006FF01FFCDE
:101AA000130760006FF09FFB97870300938787E31E
:101AB00003A747006300E50403A7C7006306E50426
:101AC00003A747016306E50403A7C7016306E5040E
:101AD00003A747026306E50403A7C7026306E504FC
:101AE00003A74703630AE50403A7C7036302A70428
:101AF000678000001307000013173700B387E70063
:101B000023A0070067800000130710006FF0DFFEBE
:101B1000130720006FF05FFE130730006FF0DFFD4A
:101B2000130740006FF05FFD130750006FF0DFFCFC
:101B3000130770006FF05FFC130760006FF0DFFBAE
:101B4000130101FF2324810023229100232021017E
:101B500013040500232611009384050013090600D1
:101B6000EF20100A032744049307F0FF6314F700E3
:101B700023220404032784049307F0FF6314F7006F
:101B800023240404EF20100B83278403639A0700A7
:101B9000130609009385040013054402EF208024F6
:101BA000EF20100683278404635AF004832744023D
:101BB00063860704930444026F00000283278404B1
:101BC0009387F7FF2324F404832784046358F002E7
:101BD000832744026384070213850400EF20403109
:101BE000E30E05FCEF20005E832784049387F7FF54
:101BF0002324F40483278404E34CF0FC9307F0FFD0
:101C00002324F404EF201003EF20807F8327440473
:101C1000635AF004832704016386070493040401D4
:101C20006F000002832744049387F7FF2322F40404
:101C3000832744046358F002832704016384070266
:101C400013850400EF20C02AE30E05FCEF20805727
:101C5000832744049387F7FF2322F4048327440453
:101C6000E34CF0FC9307F0FF2322F40403248100EB
:101C70008320C100832441000329010013010101D5
:101C80006F20407B63020504130101FD232E310107
:101C9000232C410123261102138A070023248102E9
:101CA0002322910223202103232A510123286101A9
:101CB00023267101930790009309070063FAE70058
:101CC000737004306F000000737004306F00000008
:101CD000130B05009384050013090600938B06007F
:101CE000930A08006302082C13050006EF305059D0
:101CF000130405006302052A13192900232855033C
:101D0000130609009305500A13850A00EF40C00925
:101D100003C70400832704031309C9FF230AE4024D
:101D200003C70400338927011379C9FF6306070E2F
:101D300083C71400A30AF40283C71400638E070C40
:101D400083C72400230BF40283C724006386070C97
:101D500083C73400A30BF40283C73400638E070AE1
:101D600083C74400230CF40283C744006386070A38
:101D700083C75400A30CF40283C75400638E070882
:101D800083C76400230DF40283C7640063860708D9
:101D900083C77400A30DF40283C77400638E070623
:101DA00083C78400230EF40283C78400638607067A
:101DB00083C79400A30EF40283C79400638E0704C4
:101DC00083C7A400230FF40283C7A400638607041B
:101DD00083C7B400A30FF40283C7B400638E070265
:101DE00083C7C4002300F40483C7C40063860702CA
:101DF00083C7D400A300F40483C7D400638E070014
:101E000083C7E4002301F40483C7E400638607006A
:101E100083C7F400A301F404930A440013850A0065
:101E2000A30104042326340323283405232A0404AD
:101E3000EFE0DF9113058401EFE05F919307A000CD
:101E4000B3873741232C040423288400232CF40077
:101E50002322840223220404232E040413860B006D
:101E600093050B0013050900EFE09F872320A400D2
:101E700063040A0023208A007370043017E901000C
:101E8000130989768327090097E4010093848477F6
:101E9000638C070003A7040083A70400832747047B
:101EA000938717002322F70417E7010013078774AD
:101EB000832707009387170097E6010023ACF6728B
:101EC00083A70400638E070E8327090017FB010018
:101ED000130B0B83639C070083A7040083A7C7022F
:101EE00063E6F90097E7010023AE877097E70100EA
:101EF0009387876E83A7070017E701001307076F13
:101F00000325C402032707009387170097E6010003
:101F100023A4F66C2324F4046376A70097E701005A
:101F200023A6A76C93054001EF80400293850A0029
:101F30003305AB00EFE01F828327090063880700A9
:101F400083A7040083A74704639C0708832709002D
:101F500013041000638A070083A7040083A7C70245
:101F600063F43701EFE0CFE2130504008320C102E0
:101F70000324810283244102032901028329C10130
:101F8000032A8101832A4101032B0101832BC10014
:101F9000130101036780000013850A00EF305046EB
:101FA0001304F0FF6FF05FFC13152600EF30502D87
:101FB000930A0500E31A05D21304F0FF6FF0DFFA6D
:101FC00097E7010023A08764032707009307100009
:101FD000630AF70217EB0100130B8B726FF01FF10E
:101FE00003A7040083A60400832747049387F7FF11
:101FF0002322F70483A74604E39A07F473600430AE
:102000006FF0DFF4130A000017EB0100130B4B6FA6
:10201000930BA00013050A0093054001EF701073A5
:10202000130A1A003305AB00EFE04FF0E3147AFF18
:1020300097EB0100938B4B7913850B00EFE00FEFCB
:1020400017EA0100130A8A7913050A00EFE00FEE80
:1020500017E501001305C579EFE04FED17E5010025
:102060001305457AEFE08FEC17E501001305C57AFB
:10207000EFE0CFEB97E7010023A4775997E7010042
:1020800023AE47576FF09FE6130101FF2324810021
:10209000232611002322910023202101130405008F
:1020A0007370043097E401009384045483A7040000
:1020B000639E07106318040097E701009387875415
:1020C00003A407001309440013050900EFE0CFF053
:1020D000832784026386070013058401EFE0CFEFB6
:1020E0009305090017E501001305C571EFE08FE6C0
:1020F00097E701009387475003A7070097E7010080
:102100009387874D83A707001307170097E6010001
:1021100023A4E64E03A704009387170097E6010067
:1021200023ACF64A630C070097E701009387874DBD
:1021300003A7070003274704631C070E83A70400B7
:10214000638A070697E701009387C74B03A7070039
:10215000630287107370043003A704006318070834
:1021600017E701001307C7498326070083A6060067
:102170006392060A1307F0FF97E6010023ACE644DA
:1021800003A704006308070203A707000327470407
:102190006302070203A7070083A6070083274704FB
:1021A0009387F7FF2322F70483A74604639407006D
:1021B000736004308320C100032481008324410024
:1021C00003290100130101016780000097E7010066
:1021D0009387474303A7070083A707008327470484
:1021E000938717002322F7046FF0DFEC83A6070024
:1021F00003A7070003A746041307170023A2E6045A
:1022000017E701001307C73F8326070083A60600D0
:10221000E38206F6032707000327C7000327C7004A
:102220000327470097E6010023A6E63A6FF05FF523
:1022300003A7070083A60700832747049387F7FFB8
:102240002322F70483A74604E39A07EE7360043061
:102250006FF0DFEE97E701009387873783A70700CA
:1022600063860700737004306F0000000324810050
:102270008320C100832441000329010013010101CF
:102280006FE00FB16304050C17E7010013078737F0
:1022900083260700930700006386A60A130101FF47
:1022A000232611002324810023229100737004301F
:1022B00097E601009386463383A70600638C0700E8
:1022C0000326070083270700832746049387170008
:1022D0002322F60483A70600930405000324450186
:1022E000638807008327070083A7470463940706D2
:1022F00097E701009387C73083A70700638C8706A1
:1023000097E701009387872F83A7070063848706D9
:1023100097E70100938747506306F40497E70100AD
:102320009387474E630CF402930710008320C1008B
:102330000324810083244100138507001301010158
:102340006780000013850700678000007370043009
:102350006F000000EF70505A6FF09FF99307400034
:102360006FF0DFFC83A7840293B7170093872700E1
:102370006FF0DFFB930720006FF05FFB737004309A
:1023800097E701009387472603A707006316070214
:102390006304050483A707000325C502638C0700B7
:1023A00097E701009387072603A707000327470441
:1023B000631C07026780000017E7010013078724EA
:1023C000832607000327070003A746041307170007
:1023D00023A2E604E31005FC17E701001307872298
:1023E000032507006FF01FFB03A7070083A6070064
:1023F000832747049387F7FF2322F70483A7460424
:10240000E39A07FA7360043067800000130101FF4C
:10241000232481001304050023261100EFE08FAB75
:102420006318040097E701009387C71D03A4070002
:102430000324C402EFE08FA98320C1001305040028
:1024400003248100130101016780000093079000BD
:1024500063F6B700737004306F000000130101FED3
:10246000232C8100232E1100232A910023282101EF
:102470002326310123244101130405007370043025
:1024800017E9010013094916832709006392071011
:102490006300041283270405638EF50A17E7010021
:1024A0001307471663F0B70283260700638E861270
:1024B000032707008324C702B3B4950093C4140014
:1024C0006F00000183240700B384844093B4140098
:1024D0000327C4026386E70E832784012328B404FC
:1024E00063C807009307A000B385B740232CB4004E
:1024F00093172700B387E7000327440197E90100FA
:102500009389092093972700B387F9006310F70494
:10251000130A440013050A00EFE00FAC97E701002F
:102520009387C70C0325C40283A7070063F6A7009F
:1025300097E7010023ACA70A93054001EF70102133
:1025400093050A003385A900EFE0CFA0638404005F
:10255000EFE00F8483270900638C070097E70100F1
:102560009387470A83A7070083A74704639E07044E
:102570008320C10103248101832441010329010136
:102580008329C100032A8100130101026780000032
:1025900097E701009387070703A7070083A70700B2
:1025A00083274704938717002322F704E31404EEDC
:1025B00097E701009387070503A407006FF09FEDDD
:1025C0002326B4026FF05FF1032481018320C1014F
:1025D00083244101032901018329C100032A8100C9
:1025E000130101026F705031930400006FF05FEE31
:1025F000630A0508130101FE232A910097E40100F4
:102600009384440083A70400232E1100232C81000F
:1026100023282101232631016388A7047370043025
:1026200017E90100130949FC83270900638C07009F
:1026300003A7040083A70400832747049387170098
:102640002322F7040327450197E701009387C71C5E
:10265000630EF702832709006388070083A704003D
:1026600083A74704639E07088320C10103248101D7
:1026700083244101032901018329C10013010102BF
:1026800067800000737004306F00000083278502AC
:1026900017E701001307C715E38EE7FAE39C07FA73
:1026A000930945001304050013850900EFE0CF925C
:1026B00097E70100938787F30325C40283A70700E8
:1026C00063F6A70097E7010023A2A7F29305400154
:1026D000EF70D00797E70100938787023385A70043
:1026E00093850900EFE00F8783A704000327C40246
:1026F00083A7C702E360F7F6EFD09FE96FF09FF57D
:10270000032481018320C1018324410103290101A4
:102710008329C100130101026F70101E63020506B8
:10272000130101FE232C8100232A9100232631016D
:1027300013040500232E110023282101EFD09FF957
:102740000327440197E701009387070D93090500CC
:1027500093040000630AF70213850900EFD01FF706
:102760008320C10103248101138504000329010191
:10277000832441018329C100130101026780000005
:10278000737004306F0000008327840217E5010096
:1027900013050506E382A7FCE39007FC97E7010019
:1027A000938707E383A707006394070697E7010071
:1027B000938747E583A707008324C40213094400D5
:1027C00083A7C70213050900B3B4F400EFE0CF807C
:1027D00097E70100938787E10325C40283A70700D9
:1027E00093C4140063F6A70097E7010023A0A7E0B5
:1027F00093054001EF70807597E70100938747F0DC
:10280000930509003385A700EFD0DFF46FF0DFF404
:1028100093058401EFD01FF46FF01FF4130101FE44
:1028200037150000232E1100232C8100232A91004C
:102830002328210123263101232441012322510190
:1028400023206101EF30C0236308052293040500B3
:1028500013050006EF30C0221304050063040526AB
:10286000371600009305500A2328950213850400AB
:10287000EF30805383240403B71700009387C7FF0A
:10288000B384F400B7474C4593879744130A440038
:10289000232AF40213050A00230C0402A3010404F2
:1028A0002326040223280404232A0404EFD01FEA69
:1028B00013058401EFD09FE99307A000232C0404A3
:1028C00093F4C4FF23288400232CF40023228402E1
:1028D00023220404232E040413060000971500008D
:1028E0009385C5EA13850400EFD09FDF2320A40061
:1028F0007370043017E90100130909CF8327090019
:1029000097E40100938404D0638C070003A70400BC
:1029100083A7040083274704938717002322F70423
:1029200017E70100130707CD8327070093871700D8
:1029300097E6010023A0F6CC83A704006388070A6A
:102940008327090097E90100938989DB639C0700CD
:1029500083A7040083A7C7026396070097E70100D7
:1029600023A287CA97E70100938707C703A7070039
:1029700097E60100938686C78327C40283A60600D4
:102980001307170017E601002328E6C42324E404F4
:1029900063F6F60017E70100232AF7C41395270012
:1029A0003305F5001315250093050A003385A900AA
:1029B000EFD05FDA832709006388070083A704004C
:1029C00083A74704639E070C8327090063840700DD
:1029D00083A70400EF20500793071000630AF51047
:1029E000631C0508737004306F00000097E7010056
:1029F00023AA87C0032707009307100097E9010067
:102A0000938909D0E310F7F6938A090017EB0100C8
:102A1000130B8BDB13850A00938A4A01EFD01FD179
:102A2000E31A5BFF17E50100130505DAEFD01FD0AD
:102A300097EA0100938A8ADA13850A00EFD01FCF44
:102A400017E501001305C5DAEFD05FCE17E50100E9
:102A5000130545DBEFD09FCD17E501001305C5DB5E
:102A6000EFD0DFCC97E7010023AC67B997E701000F
:102A700023A657B96FF01FEF8320C1010324810102
:102A800083244101032901018329C100032A810014
:102A9000832A4100032B010013010102678000001B
:102AA00003A7040083A60400832747049387F7FF46
:102AB0002322F70483A74604E39807F073600430E9
:102AC0006FF09FF0032481018320C10103290101DC
:102AD0008329C100032A8100832A4100032B0100BE
:102AE0001385040083244101130101026F3040115A
:102AF000737004309307F0FF17E70100232CF7AC45
:102B00000324810197E7010023A0A7AE8320C10120
:102B100083244101032901018329C100032A810083
:102B2000832A4100032B010097E7010023A207AC91
:102B3000130101026FD01F8B7370043097E70100FF
:102B400023A407AA6FD05F9C17E70100130747A8CB
:102B500083270700938717002320F7006780000072
:102B60007370043097E70100938707A803A7070055
:102B70006318070217E70100130787A7032507005B
:102B800083A70700638C070097E70100938787A757
:102B900003A70700032747046314070267800000A8
:102BA00017E70100130707A683260700032707007E
:102BB00003A746041307170023A2E6046FF09FFB48
:102BC00003A7070083A60700832747049387F7FF1F
:102BD0002322F70483A74604E39207FC73600430C2
:102BE00067800000130101FF2326110023248100C8
:102BF000EFD05FAE97E701009387879F03A407009C
:102C0000EFD0DFAC8320C100130504000324810052
:102C1000130101016780000097E701009387879DFA
:102C200003A5070067800000130101FD23261102A0
:102C3000232481022322910223202103232E310108
:102C4000232C4101232A51012328610123267101EC
:102C500097E701009387C79783A70700639A070642
:102C600017E701001307C79883270700938717000A
:102C700097E6010023AEF696832A0700638A0A0AC4
:102C800097E701009387079583A707009304000047
:102C900063FEFA0A97E90100938989A617EA010001
:102CA000130A4A9683270A009306100003A7C70257
:102CB00093172700B387E70093972700B389F9009C
:102CC00083A7090063F4F602930410006F0000026A
:102CD00097E701009387079183A7070093040000FB
:102CE0009387170017E70100232EF78E97E701005F
:102CF0009387078F83A7070063840700930410005E
:102D00008320C102032481021385040003290102E8
:102D1000832441028329C101032A8101832A4101BD
:102D2000032B0101832BC100130101036780000005
:102D300017E401001304C48C8327040083A7070051
:102D40006388070C737004306F00000017E4010003
:102D50001304048B97E901009389899A17EA01000B
:102D6000130A4A8A17EB0100130B4B8883270400D0
:102D700083A70700638007088327040083A7C70091
:102D800003A9C70083274900930B490013850B0053
:102D900063EAFA06EFD05FA483278902130589014D
:102DA00063840700EFD05FA38327C90203270B00CA
:102DB00093850B00139527003305F50013152500A7
:102DC0003385A9006376F70017E701002320F78217
:102DD000EFD05F9883270A000327C90283A7C702A1
:102DE000E366F7F8832704009304100083A7070025
:102DF000E39407F89307F0FF17D70100232CF77C23
:102E00006FF05FEA17D701002326F77C6FF09FE988
:102E100017D701001307877E8327040003270700C5
:102E200097D6010023AEE67C17D701002328F77C54
:102E300097D701009387877A83A7070093871700A6
:102E400017D70100232CF7788327040083A70700F6
:102E5000639A07009307F0FF17D70100232CF7763A
:102E60006FF01FE28327040083A7C70083A7C70072
:102E700083A7470017D70100232EF7746FF05FE098
:102E800097D701009387C77403A70700631607004D
:102E9000737004306F000000130101FE232E110037
:102EA000232C8100232A910023282101232631018C
:102EB0002324410123225101232061017370043036
:102EC00097D401009384447203A70400631007128F
:102ED00003A707001307F7FF97D6010023AAE66EA2
:102EE00083A70700639E070A97D70100938787701F
:102EF00083A707006386070A97EA0100938A4A803E
:102F000017DA0100130A8A6E17D901001309896FB5
:102F1000930910006F00C0013385EA00EFD09F8352
:102F2000832709000327C40283A7C7026374F70637
:102F300083A70A0F6380070E83A7CA0F03A4C700E5
:102F400013058401EFD05F89130B440013050B00B8
:102F5000EFD09F888327C40283260A0093050B00C5
:102F6000139527003305F5001315250013070500F9
:102F70003385AA00E3F2F6FA17D701002328F76693
:102F8000EFD04FFD832709000327C40283A7C702A0
:102F9000E360F7FA97D7010023A437656FF05FF974
:102FA0001304000083A70400638C070097D7010077
:102FB0009387476583A7070083A74704639807049F
:102FC000130504008320C1010324810183244101EE
:102FD000032901018329C100032A8100832A4100BA
:102FE000032B0100130101026780000017D70100C5
:102FF00013074761832607000327070003A746043A
:103000001307170023A2E6046FF09FECEF70C00EC9
:103010006FF01FFB17D401001304C45C8327040066
:10302000638C0702832704001309100063860702DC
:10303000EFF09FBF6306050097D7010023A2275B2F
:10304000832704009387F7FF17D70100232CF75835
:1030500083270400E39E07FC97D701009387475816
:1030600003A7070093071000E31CF7F2EFD04FD23D
:10307000130410006FF01FF363040502639605004C
:10308000737004306F00000017D701001307475416
:1030900083270700638A0700737004306F00000005
:1030A000737004306F000000130101FF23248100BE
:1030B00023261100832607000327050093861600A8
:1030C00017D601002326D65097D601009386465284
:1030D00083A606003304B7002320850063F0E604CE
:1030E0006372E40263F0860297D7010093878751E9
:1030F00003A5070013054500EFD00FEE13050400EC
:10310000EF601077EFF0DFD7630E05008320C1007A
:10311000032481001301010167800000E366E4FCE1
:103120006FF05FFC032481008320C10013010101C3
:103130006FD00FC6630E050017D70100130747496C
:103140008327070063880700737004306F00000056
:103150006FD00FC4130101FF232611002324810027
:1031600003270700930705001307170097D60100F0
:1031700023A0E64697D601009386C64817D70100DC
:10318000130707470327070003A506003304F700CA
:1031900013054500EFD04FE413050400EF60506DB8
:1031A000EFF01FCE631A0500032481008320C100C5
:1031B000130101016FD0CFBD8320C1000324810022
:1031C0001301010167800000130101FF2324810026
:1031D0002326110097D701009387873F83A7070015
:1031E000130400009387170017D701002322F73E2E
:1031F00097D701009387074083A7070063EEF51474
:1032000017DE0100130E8E5B97D201009382824E6F
:103210001304000013070000930F10001303500A5B
:103220006F00C000130ECEFE6384C20F83278EFF93
:1032300093060700E38807FE8327CEFF83A7470096
:10324000232EFEFE6386C71303AFC70083A7470084
:103250003307E500930E0000232EFEFE6380C709AE
:1032600083A8C70093874803232017012322F70070
:1032700083A788042326F7012324F70083A7C80225
:103280002328F70083A70805232C0700232AF7002B
:1032900003A808038347080063986704930708009E
:1032A0009387170083C60700B3850741E38A66FE4C
:1032B00093D525009395050193D50501231EB700ED
:1032C000938E1E0013070702630A1F038327CEFF96
:1032D00083A74700232EFEFEE394C7F983274E0001
:1032E000232EFEFE6FF0DFF793050000231EB700CC
:1032F000938E1E0013070702E31A1FFD3304D40147
:1033000013175400130ECEFE93060700E390C2F38A
:1033100097D701009387C72E03AE070083270E00BF
:103320006396071297D701009387472D03AE0700D6
:1033300083270E00639A071C17DE0100130E4E3C14
:1033400083274E10639C070283278E11639C0726F8
:103350006304060023200600EFF09FB2130504006B
:103360008320C10003248100130101016780000054
:1033700083274E00232EFEFE6FF01FED83278E1055
:1033800017DF0100130F8F4883A7470017D70100ED
:10339000232CF7466386E73D83A2C70083A7470037
:1033A000B306D500930E000017D70100232EF74473
:1033B000930F40001303500A6382E70983A8C700F4
:1033C0009387480323A0160123A2F60083A788044D
:1033D00023A6F60123A4F60083A7C80223A8F600BB
:1033E00083A7080523AC060023AAF60003A8080358
:1033F00083470800639A6732930708009387170092
:1034000003C70700B3850741E30A67FE93D725008A
:103410009397070193D70701239EF600938E1E0012
:1034200093860602638C123183278E1083A7470090
:1034300017D70100232AF73CE392E7F983270E11FF
:1034400017D701002322F73C6FF05FF783274E0068
:10345000130F8E0083A647002322DE006380E6332D
:10346000B307E50003A7460083A2C600930E000041
:103470002322EE00930F20001303500A6300EF088D
:103480008328C7001387480323A0170123A2E7005E
:1034900003A7880423A6F70123A4E70003A7C80213
:1034A00023A8E70003A7080523AC070023AAE70029
:1034B00003A8080303470800631E672213070800D8
:1034C0001307170083460700B3050741E38A66FE2A
:1034D00013D725001317070113570701239EE70091
:1034E000938E1E00938707026380122383264E006B
:1034F00003A746002322EE00E314EFF80327CE00D3
:103500002322EE006FF0DFF783274E00130F8E00AB
:1035100083A747002322FE00638CE72583A2C70010
:1035200083A74700B306D500930E00002322FE00B8
:10353000930F20001303500A6300FF0883A8C700FD
:103540009387480323A0160123A2F60083A78804CB
:1035500023A6F60123A4F60083A7C80223A8F60039
:1035600083A7080523AC060023AAF60003A80803D6
:103570008347080063986714930708009387170030
:1035800003C70700B3850741E30A67FE93D7250009
:103590009397070193D70701239EF600938E1E0091
:1035A00093860602638A121383274E0083A747007F
:1035B0002322FE00E314FFF88327CE002322FE001F
:1035C0006FF0DFF78327CE1197DE0100938E4E2533
:1035D00083A7470017D701002322F724638AD71750
:1035E00083AFC70083A747003307D500130300004C
:1035F00097D6010023A4F622130F30009302200077
:103600009308500A6388D70903A5C70093074503A9
:103610002320A7002322F700832785042326E70120
:103620002324F7008327C5022328F7008327850278
:10363000638407002326570083270505232C0700F2
:10364000232AF7000328050383470800639C170516
:10365000930708009387170083C60700B3850741C7
:10366000E38A16FF93D725009397070193D70701A5
:10367000231EF7001303130013070702638EAF0224
:103680008327CE1183A7470097D6010023A8F618F9
:10369000E39CD7F783274E1297D6010023A0F61894
:1036A0006FF09FF693070000231EF700130313002B
:1036B00013070702E396AFFC33046400E31C06C85B
:1036C0006FF09FC993070000239EF600938E1E00A3
:1036D00093860602E39A12ED17DE0100130E4E02E6
:1036E00083274E103304D40193165400E38E07C48D
:1036F0006FF0DFC813070000239EE700938E1E00C3
:1037000093870702E39412DF97D70100938707EFAF
:1037100003AE07003304D4019316540083270E0030
:10372000E38C07C06FF05FDE93070000239EF60076
:10373000938E1E0093860602E39812CF83278E1184
:103740003304D40193165400E38407C06FF09FE75D
:1037500083274E1217D701002322F70C6FF05FE882
:1037600083270E1117D701002320F70A6FF0DFC25D
:103770008327CE002322FE006FF05FDA8326CE007F
:103780002322DE006FF0DFCD130101FD2322910221
:1037900023202103232E3101232C4101232A51010F
:1037A000232861012326710123261102232481028B
:1037B00097D901009389C9E117D90100130949F488
:1037C00017DA0100130A4AE297DA0100938A8AE3C2
:1037D00097DB0100938B0BE297D401009384C4E143
:1037E000130B10006F00000283A709000324491087
:1037F0009387170017D70100232CF7DCEFF04FE871
:10380000631E040083A70400E39007FE83270900DA
:10381000E37AFBFEEFC0DFD76FF0DFFE737004309A
:1038200083270A00639E07048327091103A4C700A6
:1038300013054400EFC05FFA83A70B009387F7FFDF
:1038400017D701002328F7DA83A704009387F7FF2F
:1038500017D701002322F7DA83270A0063880700BD
:1038600083A70A0083A7470463980702032504037C
:10387000EF20003913050400EF2080386FF09FF827
:1038800003A70A0083A70A0083274704938717002A
:103890002322F7046FF05FF903A70A0083A60A004A
:1038A000832747049387F7FF2322F70483A746045F
:1038B000E39E07FA736004306FF05FFB97D7010057
:1038C000938707D183A70700639E070E130101FFAB
:1038D00023261100232481002322910097D7010081
:1038E00023A007D017D701001307C7D183270700EC
:1038F000B7A6A5A59386565A83A7070383A50700F5
:10390000639ED50003A64700631AB60083A687000E
:103910006396C60083A7C700638AD7000325070004
:103920008325070093854503EF30007717D7010003
:103930001307C7CB8326070017D40100130444DC08
:103940006F000002832707006386070883270700AC
:103950009387F7FF97D6010023AAF6C883260700AE
:1039600093972600B387D70093972700B307F400F7
:1039700083A70700E38807FC0325070093172500AA
:10398000B387A700939727003307F40083264700E7
:1039900093878700B307F40083A44600232297008F
:1039A000638EF40283A7C4008320C1000324810036
:1039B00017D701002328F7C4832441001301010114
:1039C000678000009307100017D70100232AF7C073
:1039D00067800000737004306F00000083A444000F
:1039E00093054001EF6080563305A4002322950023
:1039F0006FF05FFB130101FE23282101232E11002C
:103A0000232C8100232A910023263101130905006C
:103A10007370043097D40100938404BD83A704001D
:103A200017D40100130404BE639C070C631409003F
:103A3000032904009309490013850900EFC0DFD969
:103A4000832789026386070013058901EFC0DFD849
:103A50009385090017D50100130505DCEFC09FCF42
:103A600083A70400638807008327040083A7470413
:103A70006394070A832704006384270D83A7040047
:103A8000638207067370043083A704006398070EEF
:103A900097D701009387C7B603A70700032707003E
:103AA0006310070C9307F0FF17D701002324F7B228
:103AB00083A70400638807028327040083A74704C1
:103AC0006382070203270400832604008327470438
:103AD0009387F7FF2322F70483A746046394070024
:103AE000736004308320C1010324810183244101D8
:103AF000032901018329C10013010102678000002D
:103B000003270400832704008327470493871700B3
:103B10002322F7046FF09FF103270400832604009B
:103B2000832747049387F7FF2322F70483A74604DC
:103B3000E39207F47360043083270400E39027F5D1
:103B400083A704006382070697D70100938747A8DD
:103B500083A707006388070A737004306F000000B2
:103B600083A7070083A7C70083A7C70083A74700D1
:103B700017D701002320F7A66FF09FF30327040057
:103B80008327040083274704938717002322F70421
:103B900097D701009387C7A603A70700032707004D
:103BA000E30207F06FF0DFFB97D70100938787A44C
:103BB00017D701001307C7B483A70700032787118E
:103BC0006314F7028320C1010324810197D7010008
:103BD00023AA07A283244101032901018329C100EB
:103BE0001301010267800000032481018320C101C9
:103BF00083244101032901018329C100130101022A
:103C00006FF0DFCB032481018320C10183244101B4
:103C1000032901018329C100130101026FC05F97CD
:103C20006306050A130101FF2322910097D40100C6
:103C30009384449D232021011389050083A504005A
:103C4000232611002324810093858501EFC09FB3B3
:103C500003A5040013054500EFC01FB89307F0FF4C
:103C6000630AF90697D701009387879803A4070092
:103C700003A7040083A7070033042401232287003D
:103C8000636EF40697D701009387879703A5070013
:103C900083A5040093854500EFC0DFAE97D70100F0
:103CA0009387479383A707006376F40097D70100B3
:103CB00023A287928320C100032481008324410032
:103CC00003290100130101016780000073700430B3
:103CD0006F00000083A50400032481008320C1003D
:103CE000832441000329010017D501001305C5B243
:103CF00093854500130101016FC0DFA597D701002F
:103D00009387C78F03A507000324810083A50400C0
:103D10008320C100832441000329010093854500CD
:103D2000130101016FC01FA6630E050097D70100A4
:103D30009387078A83A70700639A0700737004308C
:103D40006F000000737004306F000000130101FF6A
:103D50002322910097D401009384C48A03A704000E
:103D60009387050083A50400B7060080B3E7D7005A
:103D70002326110023248100232CF700938585013D
:103D800013040600EFC01F9D03A5040013054500A2
:103D9000EFC09FA49307F0FF6304F40297D70100DC
:103DA0009387078503A507008320C1008324410072
:103DB0003305850003248100130101016F60402B4E
:103DC00083A50400032481008320C10083244100D3
:103DD00017D50100130545A4938545001301010182
:103DE0006FC05F976308050A130101FF232291004A
:103DF00097D40100938404812320210113890500B5
:103E000083A50400232611002324810093858501C6
:103E100013040600EFC01F9403A50400130545001A
:103E2000EFC09F9B93071000630AF40697C7010039
:103E30009387077C03A4070003A7040083A7070058
:103E40003304240123228700636EF40697C7010020
:103E50009387077B03A5070083A50400938545008E
:103E6000EFC05F9297C701009387C77683A70700CB
:103E70006376F40097C7010023AE87748320C100E6
:103E8000032481008324410003290100130101015F
:103E900067800000737004306F00000083A5040089
:103EA000032481008320C1008324410003290100F1
:103EB00017D50100130545969385450013010101AF
:103EC0006FC05F8997C701009387477303A50700F9
:103ED0000324810083A504008320C10083244100C2
:103EE0000329010093854500130101016FC09F89DB
:103EF000130101FF232611002324810023229100B6
:103F00008327C50003A4C7006304040A9304840143
:103F100013850400EFC05F8C97C701009387476B40
:103F200083A70700639A07089304440013850400DD
:103F3000EFC09F8A97C701009387476B0327C4028E
:103F400083A7070063F6E70097C7010023A0E76A8D
:103F500093172700B387E7009397270017C5010041
:103F60001305057A938504003305F500EFC08FFE35
:103F700097C701009387076983A707000327C40237
:103F80001305000083A7C70263FAE7009307100038
:103F900017C701002326F764130510008320C10012
:103FA0000324810083244100130101016780000084
:103FB000737004306F0000009385040017D5010072
:103FC00013050583EFC00FF96FF09FFA97C7010043
:103FD0009387076083A70700639607007370043018
:103FE0006F000000130101FF23261100232481002C
:103FF00023229100B70700800324C500B3E7F50032
:104000002320F50063080408EFC00FFD930444006B
:1040100013850400EFC04FFC97C701009387075D2D
:104020000327C40283A7070063F6E70097C70100D0
:1040300023AEE75A93172700B387E700939727002B
:1040400017C501001305C56B3305F5009385040002
:10405000EFC04FF097C701009387C75A83A70700A7
:104060000327C4021305000083A7C70263FAE70011
:104070009307100017C701002324F75613051000FB
:104080008320C10003248100832441001301010126
:1040900067800000737004306F0000006304050245
:1040A00097C701009387875303A7070097C70100AD
:1040B0009387075483A707002320E5002322F500F8
:1040C00067800000737004306F0000006304050E09
:1040D000638E050C130101FF2326110023248100A8
:1040E000130705007370043097C801009388C84F08
:1040F00083A708006380070297C701009387875052
:1041000083A6070083A7070083A7460493871700A9
:1041100023A2F60417C301001303834D83A70500F0
:10412000032603009306F0FF130400006388D704FE
:1041300017CE0100130E8E4A03250E000328070038
:10414000832647006306A800130410006378D60294
:104150003308D640130410006372F80203250E00E2
:10416000B387C74003260300B387D70023A0F50019
:104170002320A7002322C7001304000083A7080000
:10418000638C070097C701009387C74783A7070081
:1041900083A7470463940702130504008320C1002A
:1041A0000324810013010101678000007370043053
:1041B0006F000000737004306F000000EF50D07388
:1041C0006FF09FFD9307100017C70100232AF740E7
:1041D00067800000630605000325C50467800000B2
:1041E0001305000067800000630405002326B50462
:1041F0006780000097C701009387C74003A50700A9
:104200006780000097C701009387073E83A70700D8
:1042100013051000638C070097C701009387473B85
:1042200003A507001335150013151500678000005E
:10423000630C0508130101FE232A910097C40100B5
:104240009384443C83A70400232E1100232C810077
:1042500023282101232631010327C50283A7C70292
:104260006376F7048327850163CC070083A70400E6
:1042700083A6C7029307A000B387D740232CF5007D
:1042800093172700B387E7000327450117C90100EB
:104290001309094793972700B307F9006308F7024A
:1042A00083A7040083A7C7022326F5028320C10148
:1042B0000324810183244101032901018329C100D1
:1042C0001301010267800000678000009309450028
:1042D0001304050013850900EFC00FD083A7040065
:1042E00017C70100130787300327070083A7C702FA
:1042F0002326F4026376F70017C701002328F72E60
:10430000139527003305F5000324810113152500BB
:104310008320C10183244101938509003305A9004D
:104320008329C10003290101130101026FC08FC25B
:1043300063060502130101FF2326110023248100D7
:104340002322910097C701009387C72B03A407007E
:10435000630AA400737004306F00000013050000AE
:10436000678000008327440563960700737004305C
:104370006F0000008326C402032704059387F7FF1C
:10438000232AF4046384E600638E0700130500000B
:104390008320C10003248100832441001301010113
:1043A000678000009304440013850400EFC0CFC26F
:1043B0000325040597C701009387472303A7070038
:1043C0009307A000B387A7402326A402232CF40060
:1043D0006376A70097C7010023AAA7209305400191
:1043E000EF50D03697C70100938787313385A700F8
:1043F00093850400EFC00FB6130510006FF05FF94E
:104400007370043097C701009387071E83A70700C6
:104410006380070297C701009387C71E03A70700A1
:1044200083A7070083274704938717002322F704F5
:104430006780000097C701009387071B83A70700C9
:10444000638C070297C701009387C71B03A7070068
:10445000032747046302070203A7070083A6070098
:10446000832747049387F7FF2322F70483A7460493
:1044700063940700736004306780000097C70100F1
:104480009387471803A6070083A6070003A7070022
:104490009307A00083A6C60203258601B387D740F1
:1044A000232CF7006780000097C7010093878715CA
:1044B00003A70700630A070083A6070003A74605B2
:1044C0001307170023AAE60403A50700678000006E
:1044D000130101FD2320210323261102232481023D
:1044E00023229102232E3101130905007370043039
:1044F00097C401009384440F83A7040017C40100EC
:1045000013044410639E070A8327040083A78705CA
:10451000639A0700832704001307100023AEE70403
:10452000639A050E83A704006388070083270400AD
:1045300083A74704639A07147370043083A70400A9
:10454000639407068327040003A587056308050015
:10455000630209048327040023AC070483270400B3
:1045600023AE070483A704006388070083270400A1
:1045700083A74704639207068320C10203248102B4
:1045800083244102032901028329C101130101038C
:104590006780000003270400832787059387F7FFC0
:1045A000232CF7046FF09FFB0327040083270400EC
:1045B00083274704938717002322F7046FF09FF89F
:1045C00003270400832704008327470493871700E9
:1045D0002322F7046FF05FF303270400832604000F
:1045E000832747049387F7FF2322F70483A7460412
:1045F000E39407F8736004308320C102032481022E
:1046000083244102032901028329C101130101030B
:1046100067800000032504002326B1001305450030
:10462000EFC08F9B8325C1009307F0FF6380F508DF
:1046300097C701009387C7FB83A9070003270400DE
:1046400083A70700B389B9002322370163ECF90679
:1046500097C701009387C7FA03A5070083250400C5
:1046600093854500EFC00F9297C70100938787F6A7
:1046700083A7070063F6F90097C7010023AC37F55D
:10468000EFB01FF16FF01FEA032704008326040038
:10469000832747049387F7FF2322F70483A7460461
:1046A000E39C07E8736004306FF01FE98325040082
:1046B00017C501001305451693854500EFC08F8986
:1046C0006FF01FFC97C70100938747F303A507000E
:1046D0008325040093854500EFC0CF8A6FF05FFA11
:1046E000130101FD23202103232E31012326110272
:1046F0002324810223229102232C410113890500E6
:10470000930906007370043097C401009384C4EDCC
:1047100083A7040017C401001304C4EE639C0714AC
:1047200003270400930720000327C7056304F7024B
:10473000832704001345F5FF03A787053375E500BC
:1047400023ACA704832704001307100023AEE7045B
:10475000639A060A83A7040063880700832704007E
:1047600083A74704639407167370043083A704007B
:10477000639E0706638809008327040083A78705D3
:1047800023A0F9000327040093071000130500007D
:104790000327C705630EF700832704001349F9FFB9
:1047A0001305100003A787053379E90023AC27051B
:1047B0008327040023AE070483A70400638807004F
:1047C0008327040083A747046392070C8320C10258
:1047D0000324810283244102032901028329C101A8
:1047E000032A8101130101036780000003270400ED
:1047F0008327040083274704938717002322F704A5
:104800006FF05FF7032504002326D1001305450050
:10481000EFB09FFC8326C1009307F0FF638AF60C7C
:1048200097C701009387C7DC03AA0700032704008A
:1048300083A70700330ADA00232247016368FA0CD2
:1048400097C701009387C7DB03A5070083250400F2
:1048500093854500EFB01FF397C70100938787D773
:1048600083A707006370FA0A97C7010023A447D7FC
:104870006F004009032704008327040083274704AF
:10488000938717002322F7046FF09FE903270400A2
:1048900083260400832747049387F7FF2322F70426
:1048A00083A74604E39407F2736004308320C102B7
:1048B0000324810283244102032901028329C101C7
:1048C000032A81011301010367800000032704000C
:1048D00083260400832747049387F7FF2322F704E6
:1048E00083A74604E39207E8736004306FF0DFE7C4
:1048F0008325040017C50100130505F293854500C3
:10490000EFB05FE5EFB0DFC86FF0DFE497C70100FD
:104910009387C7CE03A50700832504009385450030
:10492000EFB05FE66FF01FFE630A050C130101FF95
:10493000232611002324810023229100232021011A
:104940007370043097C40100938404CA83A70400E1
:1049500063960708638606008327850523A0F60073
:1049600093070600930620000326C505232ED504D1
:1049700013870500130405006382D70A63F4F60861
:10498000930530006388B700930540006396B70035
:10499000630CD610232CE40493071000630CF60874
:1049A0001304100083A70400638C070097C701005D
:1049B000938747C583A7070083A747046398070623
:1049C000130504008320C1000324810083244100D7
:1049D00003290100130101016780000097C701004E
:1049E000938747C203A7070083A7070083274704CD
:1049F000938717002322F7046FF0DFF573700430FC
:104A00006F00000093061000E398D7F88327850510
:104A100033E7B700232CE5046FF01FF883278505E3
:104A200093871700232CF5046FF01FF7EF50C06C2D
:104A30006FF01FF91309440013050900EFB0DFD927
:104A400097C70100938787BA0325C40283A707008D
:104A500063F6A70097C7010023AAA7B893054001F2
:104A6000EF50C04E97C70100938787C93385A700D1
:104A700093050900EFB01FCE8327840263860700E9
:104A8000737004306F00000097C70100938787B7E9
:104A900083A707000327C40283A7C702E3F2E7F056
:104AA000EFB01FAF6FF0DFEF130400006FF09FEF68
:104AB00063080508130101FE232C8100232A9100BD
:104AC00023282101232631012324410123225101DE
:104AD000232E110093090700138A06009304060091
:104AE0001389050013040500EFB0DFBE930A05002B
:104AF00063060A00832784052320FA000327C405E0
:104B000093072000232EF4046380F40463FA9710C3
:104B1000930630006388D400930640006396D40067
:104B2000630CF70E232C2405930710006312F70A79
:104B30008327840263820702737004306F000000D1
:104B4000737004306F00000083278405938717007B
:104B5000232CF4046FF05FFD97C70100938747A7EC
:104B600083A707006390070A930444001385040099
:104B7000EFB09FC697C70100938747A70325C402DC
:104B800083A7070063F6A70097C7010023A0A7A685
:104B900093054001EF50803B97C70100938747B6CC
:104BA000938504003385A700EFB0DFBA97C70100F3
:104BB000938747A583A707000327C40283A7C702DB
:104BC00063F8E700638609009307100023A0F9004B
:104BD0001304100013850A00EFB05FAF1305040043
:104BE0008320C101032481018324410103290101A0
:104BF0008329C100032A8100832A41001301010295
:104C0000678000009305840117C50100130545BEA8
:104C1000EFB05FB46FF09FF9130400006FF09FFBDB
:104C200093071000E392F4F08327840533E927010A
:104C3000232C24056FF05FEF630A050E130101FEBC
:104C4000232C8100232A910013040500232631011F
:104C5000232E11002328210193840500EFB09FA784
:104C6000930720008326C405232EF404832784059C
:104C7000130710009309050093871700232CF404F1
:104C80006396E60883278402638607007370043006
:104C90006F00000097C701009387879383A70700E1
:104CA000639A07081309440013050900EFB0DFB247
:104CB00097C70100938787930325C40283A7070042
:104CC00063F6A70097C7010023A2A79293054001AE
:104CD000EF50C02797C70100938787A2930509006B
:104CE0003385A700EFB01FA797C70100938787916F
:104CF00083A707000327C40283A7C70263F8E7005E
:104D0000638604009307100023A0F40003248101AC
:104D10008320C10183244101032901011385090076
:104D20008329C100130101026FB05F9A73700430D0
:104D30006F0000009305840117C50100130545AB02
:104D4000EFB05FA16FF05FFA9307050063080506F7
:104D50007370043017C70100130707898326070003
:104D6000639E060203A6C7059306200013050000F4
:104D70006316D60023AE070413051000832707002F
:104D8000638C070097C701009387C78703A70700B5
:104D900003274704631C07026780000097C60100D1
:104DA0009386468603A6060083A60600832646044D
:104DB000938616002322D6046FF0DFFA97C701000E
:104DC0009387478483A707006FF09FF803A7070026
:104DD00083A60700832747049387F7FF2322F7045E
:104DE00083A74604E39A07FA7360043067800000E3
:104DF000130101FB2322910423202105232C4103CD
:104E0000232A510323286103232671032326110437
:104E100023248104232E310323248103232291039D
:104E20002320A10317B901001309C97E17BB010094
:104E3000130B8B7D97B401009384447D97BA0100D6
:104E4000938A0A7D130A1000930B900083270900B0
:104E500003A707006306071683A7C70083A90700F7
:104E6000EFD09FCEEFD0DFCF83270B00130C0500D0
:104E70006368F50C97B7010023A8A7781306000014
:104E80006376352303A50400B3858941EFC05FCB6A
:104E9000EFD01FFF6306051603A50400930600006C
:104EA0001306000093058100EFC0CFC9E30005FAA7
:104EB00083278100E3C207FE8329010183A74901FB
:104EC0006386070013854900EFB01F91EFD05FC9DB
:104ED00083270B00130C05006362F50C8327810008
:104EE00017B7010023228773E3E8FBFAB317FA0030
:104EF00013F707216310072013F7770C6316072AAF
:104F000093F70702E38A07F813850900EF00504F73
:104F10006FF09FF883A7C70003A4C70083AC070006
:104F20009309440013850900EFB01F8B83274402C7
:104F300013050400E78007008327C4016386470D3B
:104F40008327090003A70700E31607FC03A70A004D
:104F500097B6010023AA866B97B6010023AAF66ACA
:104F600097B7010023A8E76AEFD09FF16FF0DFF257
:104F700083A7C70003A4C70003AD0700930C440038
:104F800013850C00EFB05F858327440213050400EE
:104F9000E78007008327C401638C470B8327090040
:104FA00003A70700E31607FC03A70A0097B6010052
:104FB00023A0F66697B7010023AEE7646FF01FF2F7
:104FC000EFD09FB8EFD0DFB983270B00130C05009B
:104FD000E368F5F683A70A0003A50400930900001F
:104FE00003A60700B385894117B70100232E876107
:104FF00013361600EFC0DFB4EFD09FE8E31E05E8DC
:10500000EFB00FD96FF05FE9832784019385090022
:10501000B387FC0063E2FC0883A7040063860702F1
:10502000232A0100232C9101232E8100EFF08F9D74
:1050300003A5040093060000130600009305410138
:10504000EFB0DFB0E31E05EE737004306F000000B8
:105050008327840193850C00B307FD006362FD087C
:1050600083A7040063860702232A0100232CA101E1
:10507000232E8100EFF00F9903A504009306000092
:105080001306000093054101EFB05FACE31805F093
:10509000737004306F000000032509002322F40020
:1050A00023288400EFB00FEE6FF09FE9EFD05FDDB3
:1050B0008327090083A7C70003A4C700930C4400FB
:1050C00013850C00EFB04FF18327C401638A4705B5
:1050D0008327440213050400E78007006FF0DFDB3D
:1050E000032509002322F40023288400EFB08FE970
:1050F0006FF0DFEA8327C10023ACF9006382070A5F
:10510000B387870123A2F90023A8390193854900B9
:105110006362FC0803A50A00EFB0CFE66FF0DFD7AB
:1051200083278401232884003387F9002322E400A5
:10513000636AEC04330C3C41636EFC0283A70400F9
:1051400063860702232A0100232C3101232E8100CC
:10515000EFF04F8B03A50400930600001306000038
:1051600093054101EFB09F9EE31405F67370043080
:105170006F00000003A50A0093850C00EFB08FE0DC
:105180006FF01FF50325090093850C00EFB08FDF4A
:105190006FF01FF403250900EFB0CFDE6FF0DFCF13
:1051A000737004306F0000008327C10083A689015B
:1051B00023A839013387D70023A2E9006362EC06F4
:1051C000B307FC4063EAD70683A7490213850900A9
:1051D000E780070083A7C901E39047CD83A6890133
:1051E0008327C10003A70400B387D7006306070223
:1051F000232A0100232CF100232E3101EFF08F80B0
:1052000003A5040093060000130600009305410166
:10521000EFB0DF93E31205C8737004306F00000035
:105220006374FC00E372F7FA0325090093854900D3
:10523000EFB04FD56FF05FC603A50A009385490014
:10524000EFB04FD46FF05FC5130101FF232481003D
:1052500023261100232291002320210117B40100ED
:105260001304C43AEFF0CF99832704006384070442
:10527000EFF04F9C83270400638A07029308000025
:105280001308000093070000130720009306000096
:105290001306004097B501009385C5191705000056
:1052A000130545B5EFC01F9E6314050673700430E7
:1052B0006F00000017B901001309495713050900D1
:1052C000EFB0CFC697B401009384845713850400D0
:1052D000EFB0CFC5130600009305C00013054000D2
:1052E00097B7010023A8273397B7010023A297326D
:1052F000EFB08FF117B70100232AA730630605022C
:1053000097B5010093858512EFC04FF06FF05FF6FF
:105310008320C1000324810083244100032901006C
:105320001301010167800000737004306F000000FA
:10533000638A050A130101FD232A5101930A05001E
:105340001305C0022324810223229102232021037A
:10535000232E3101232C4101232611022328610130
:10536000232671011309070093890600130A06001A
:1053700093840500EF00C07013040500630C050260
:10538000EFF00F8897B701009387472883A707009E
:10539000638E0704EFF00F8A1305440023205401A5
:1053A000232C9400232E440123203403232224039E
:1053B000EFB0CFB9130504008320C102032481029A
:1053C00083244102032901028329C101032A8101A7
:1053D000832A4101032B0101832BC1001301010327
:1053E00067800000737004306F00000097BB0100FD
:1053F000938BCB4313850B00EFB04FB317BB01006A
:10540000130B0B4413050B00EFB04FB21306000053
:105410009305C0001305400097B7010023AC771F28
:1054200097B7010023A6671FEFB00FDE17B7010083
:10543000232EA71C630A050097B50100938505FF7D
:10544000EFC0CFDC6FF01FF5737004306F00000009
:10545000630E0506130101FE232C8100232E11008B
:10546000232A910017B401001304441A832804006E
:105470001308050013050000638008049304070067
:105480002322B100138706002324C1002326010133
:105490009306500063C0B604EFE0DFD69307200008
:1054A000630EF504032504009306000013060000B4
:1054B00093054100EFB08FE98320C10103248101EE
:1054C00083244101130101026780000073700430DE
:1054D0006F000000930541009306000013060700CB
:1054E00013850800EFB05FB88320C1010324810158
:1054F0008324410113010102678000000325040099
:10550000930600001386040093054100EFB00FE4FA
:105510006FF09FFA63060500032505006780000011
:10552000737004306F000000631605007370043060
:105530006F000000130101FF2326110023248100C6
:1055400013040500EFE0DFEB032544013334A00032
:10555000EFE05FEE130504008320C1000324810007
:1055600013010101678000006316050073700430A9
:105570006F000000130101FF2324810013040500C4
:1055800023261100EFE0DFE703240402EFE09FEAA7
:105590008320C100130504000324810013010101CD
:1055A0006780000063160500737004306F00000010
:1055B000130101FF2324810023229100138405009D
:1055C0009304050023261100EFE09FE323A084024B
:1055D000032481008320C1008324410013010101C1
:1055E0006FE05FE5130101FF1305C0012324810073
:1055F00023261100EF00C0481304050063080500CE
:105600002320050013054500EFB04F921305040059
:105610008320C10003248100130101016780000081
:1056200063020502B70700FFB3F7F50063860700C2
:10563000737004306F000000639A050073700430CB
:105640006F000000737004306F000000130101FE52
:10565000232C810023282101232631012324410109
:1056600023225101232E1100232A910093090700C0
:1056700013890600930A060013840500130A050027
:10568000EFE05FB8631805006386090073700430AB
:105690006F000000EFD04FCB83240A00B377940053
:1056A000631209046382070463880A009347F4FFC6
:1056B000B3F797002320FA00EFD08FFC8320C101BD
:1056C000032481011385040003290101832441017E
:1056D0008329C100032A8100832A410013010102AA
:1056E00067800000E302F4FCE38809FCB335500155
:1056F0009395850163060900B7070004B3E5F5003B
:1057000013860900B3E5850013054A00EFE0CFE1F9
:10571000EFD00FF763140500EFA09FE7EFE01FD66F
:10572000931765009309050063DA0700B7040001C9
:105730009384F4FFB3F499006FF05FF8EFE05FCC6F
:1057400083290A00B377340163100902638A0700D2
:1057500063880A009347F4FFB3F737012320FA0068
:10576000EFE05FCD6FF09FFCE31CF4FE6FF05FFE97
:10577000630C0500B70700FFB3F7F500638A070065
:10578000737004306F000000737004306F0000000D
:10579000130101FF232481001304050023261100B7
:1057A000232291002320210113890500EFE05FC52A
:1057B000832404009345F9FFB3F795002320F400F8
:1057C000EFE05FC78320C10003248100138504003C
:1057D00003290100832441001301010167800000B7
:1057E000130101FF23248100130405002326110067
:1057F000EFA05FEE03240400EFA05FED8320C10063
:1058000013050400032481001301010167800000D7
:10581000630C0500370700FFB3F7E500638A070054
:10582000737004306F000000737004306F0000006C
:105830006F40500FB70700FFB377F600638607008D
:10584000737004306F00000063160600737004303C
:105850006F000000130101FE232C81002328210189
:105860002326310123244101232E1100232A9100F4
:105870001389060093890500130A05001304060026
:10588000EFE05F98631E050463060900737004303F
:105890006F000000EFD04FAB83240A00938509000E
:1058A00013050A00B3E49900EFF09FF6B377940074
:1058B000630AF40883240A00EFD08FDC8320C1013F
:1058C000032481011385040003290101832441017C
:1058D0008329C100032A81001301010267800000AF
:1058E000EFD08FA683240A009385090013050A00D0
:1058F000B3E43401EFF0DFF1B3F78400638487048D
:10590000E30A09FAB705000513060900B365B400F8
:1059100013054A00EFE04FC1EFD08FD663140500A6
:10592000EFA01FC7EFE09FB5931765009304050034
:1059300063D40702B70700019387F7FFB3F4F400BD
:105940006FF0DFF783270A001344F4FFB3F78700F3
:105950002320FA006FF05FF6EFE09FAA83240A008D
:10596000B3779400639887009347F4FFB3F79700E9
:105970002320FA00EFE01FAC6FF0DFFB130101FF03
:105980002324810023261100130405002322910003
:10599000EFD08F9B83274400638607020325040111
:1059A0009304C400631895006F008003032504016D
:1059B00063089502B7050002EFE04FE1832744003A
:1059C000E39607FE13050400EF0080230324810003
:1059D0008320C10083244100130101016FD04FCA0D
:1059E000737004306F000000630C0500370700FF80
:1059F000B3F7E500638A0700737004306F0000009E
:105A0000737004306F0000006F40C071630C0500BC
:105A1000B70700FFB3F7F500638A0700737004301F
:105A20006F000000737004306F000000130101FF6D
:105A30002324810023229100232611001304050052
:105A400093840500EFE0DF9B0327040093C7F4FF76
:105A5000B377F7002320F400032481008320C100E2
:105A600083244100130101016FE0DF9C6306050000
:105A70000325850167800000130500006780000092
:105A8000130101FF232481002326110013040500C4
:105A9000EFD08F8B97B70100938707B883A70700D4
:105AA000639C0704B797010017B701001307C7DA13
:105AB0009387C7FF97B6010023A6E6B617B7010084
:105AC0002320F7B617B70100232AF7D897B70100AC
:105AD0009387C7B417B701002320F7D893071000A6
:105AE00017B70100232207B417B70100232807B214
:105AF00017B701002322F7B263120402EFD04FB8A8
:105B0000EF10C05813040000130504008320C100E7
:105B10000324810013010101678000001305840044
:105B2000937735006398070CB79701001307F5FFCB
:105B30009387A7FFE3E4E7FC97B60100938686AE60
:105B400083A706006F00400103A70700630A070050
:105B5000938607009307070003A74700E366A7FEA5
:105B600017B70100130787ABE38AE7F803A707001D
:105B7000130600011384870023A0E60003A7470053
:105B8000B306A740637ED6023388A7002322D8003D
:105B900023A2A7008325480097B60100938686A814
:105BA0006F0080009306070003A706000326470046
:105BB000E36AB6FE2320E80023A0060103A74700FE
:105BC00097B701009387C7A983A70700B387E7406A
:105BD00017B701002326F7A8EFD08FAAE30204F23B
:105BE000130504008320C100032481001301010177
:105BF000678000001375C5FF130545006FF0DFF2E5
:105C000063080506130101FF2324810023261100E8
:105C100013040500EFC05FF3930584FF0326C4FF60
:105C200017B70100130707A06F0080001387070054
:105C30008327070083A64700E3EAC6FE232CF4FE71
:105C40002320B70097B70100938787A103A7070018
:105C50008327C4FF032481008320C100B387E700AA
:105C600017B70100232EF79E130101016FD04FA13A
:105C70006780000097B701009387879E03A5070000
:105C800067800000678000003367B5001377370036
:105C900093070500631207049308D6FFB3081501A4
:105CA00013070500938605006378150303A8060013
:105CB0001307470093864600232E07FFE36817FF6C
:105CC0009347F5FFB387170193F7C7FF9387470003
:105CD000B385F500B307F5003306C50063F4C70CC0
:105CE0009386450013884700B3B6D70033B8050143
:105CF00033E7F50093C616001348180013773700F2
:105D0000B3E60601133717003377D700330EF6409A
:105D100093861700630807061337AE00631407065F
:105D200013532E0013880500938607001307000005
:105D300083280800130717001308480023A0160142
:105D400093864600E36667FE1377CEFFB385E500D2
:105D5000B387E7006306EE0483C6050013871700C8
:105D60002380D700637EC70283C6150013872700F0
:105D7000A380D7006376C70203C725002381E7000D
:105D800067800000B307F640B387F50093851500E0
:105D900003C7F5FF93861600238FE6FEE398F5FE12
:105DA0006780000067800000B367C50093F7370085
:105DB000B308C5006382070E63761511B307A040D0
:105DC00093F73700138737009306500093F5F50FCC
:105DD000130815003383A8401306F6FF6374D70039
:105DE000130750006368E60E6380070E2300B500BA
:105DF00013071000638EE700A300B50013073000FF
:105E0000130825006396E700130835002301B50049
:105E10001396850033E6C500139705013367E60046
:105E20003303F34093968501B366D70013562300DE
:105E3000B307F5001307000023A0D70013071700CE
:105E400093874700E36AC7FE1377C3FFB307E800F1
:105E50006300E3082380B70013871700637C1703F0
:105E6000A380B70013872700637617032381B70049
:105E70001387370063701703A381B70013874700A8
:105E8000637A17012382B7001387570063741701E1
:105E9000A382B7006780000093F5F50F1397850084
:105EA000B365B700139705013367B700E37415FFB7
:105EB000930705009387470023AEE7FEE3EC17FF47
:105EC0006780000067800000130805006FF05FF432
:105ED00067800000930705006FF0DFF78347050038
:105EE00013070500638C07001305150083470500A1
:105EF000E39C07FE3305E5406780000013050000C2
:105F000067800000130515008347F5FF9385150092
:105F100003C7F5FF63880700E386E7FE3385E740A4
:105F200067800000930700006FF05FFF9307050094
:105F30009385150003C7F5FF93871700A38FE7FE2E
:105F4000E31807FE67800000834605009307000200
:105F50006398F6001305150083460500E38CF6FEF2
:105F6000938756FD93F7D70F6380070493070500C7
:105F7000930500006388060413050000938717004B
:105F8000138606FD1317250083C607003305A700F7
:105F9000131515003305A600E39206FE6384050081
:105FA0003305A04067800000938536FD83461500C9
:105FB00093B5150093071500E39006FC1305000048
:105FC0006FF0DFFD130500006780000083A7050068
:105FD0002380A70083A705009387170023A0F5005F
:105FE0006780000097A601009386466483A7060099
:105FF000174703001307078913861700B307F70035
:106000002380A70097A5010023A2C5629307A000E3
:10601000630AF500930700046308F6001305000007
:1060200067800000E30C06FE370610F01307170028
:106030008347F7FF2320F6F083A706009387F7FF37
:1060400097A5010023A4F55EE39207FE1305000067
:1060500067800000130101EB2322911423202115F6
:10606000232A51132324811323261114232481145A
:10607000232E3113232C411323286113232671135C
:10608000232291132320A113232EB1119304050081
:10609000138905002326C100130C5002930A9000B7
:1060A0008347090063888703638C070603A4040001
:1060B0006F008000638607062300F40003A4040039
:1060C000130919001304140023A084008347090056
:1060D000E39287FF0346190093081900938608008E
:1060E000130D00029309F0FF130AF0FF13080000DC
:1060F000130550059307D6FD93F7F70F1389160084
:10610000636EF53A17A701001307C7EF93972700AF
:10611000B387E70083A70700B387E700678007001E
:106120008320C114032481148324411403290114FE
:106130008329C113032A8113832A4113032B0113DB
:10614000832BC112032C8112832C4112032D0112C7
:10615000832DC1111301011567800000930C80008D
:10616000232401009307100063DA071D8327C10071
:1061700003A40400938B770093F68BFF03AB060018
:1061800083A94600938786002326F10013860C001E
:106190009306000013050B0093850900EF2040745F
:1061A0002328A1009307000063803733930D41013A
:1061B000930B100013860C009306000013050B00D0
:1061C00093850900EF2000149306000013860C004D
:1061D000130B050093890500EF2080708327810051
:1061E00023A0AD0093861B00938D4D00638637017D
:1061F000938B06006FF01FFCE37C9BFF63D246038A
:10620000930704002380A70103A40400130AFAFFE4
:106210009307140023A0F40013840700E3C446FF8F
:1062200093962B0093070101B386D7006F0080027D
:10623000938777052300F40003A40400938BFBFFEE
:1062400093871B001304140023A084009386C6FFC9
:10625000E358F0E483A70600E3ECFAFC9387070316
:106260006FF05FFD83A70400930600030327C100BE
:106270002380D70083A7040093064700930C0001F6
:106280001386170023A0C40013068007A380C7004D
:1062900003A404002324010093070700130414003F
:1062A00023A0840003AB0700930900002326D1003C
:1062B0006FF0DFED8327C10083AC0700938B4700AD
:1062C00063880C28635C40259307D002631EFD2081
:1062D00083C70C006388070263D8092483A60400DF
:1062E000938C1C00130AFAFF2380F60003A4040019
:1062F0001304140023A0840083C70C00E39E07FC52
:106300006352400303A40400930700022300F40037
:1063100003A40400130AFAFF1304140023A084004A
:10632000E3160AFE232671016FF09FD72324010094
:1063300093071000930CA000E3CA07E38327C10072
:1063400003A40400938647006FF0DFF503C6160030
:10635000930609006FF01FDA83A70400930650022A
:106360002380D70003A404001304140023A0840096
:106370006FF01FD3930C0001232401006FF09FDE08
:106380008327C10003C616009306090083A90700EE
:10639000938747002326F100E35E0AD4138A09009D
:1063A0009309F0FF6FF01FD503C61600130DD0023E
:1063B000930609006FF01FD49347FAFF93D7F74174
:1063C00003C61600337AFA00930609006FF09FD2D5
:1063D00003C61600130D0003930609006FF09FD14A
:1063E00083C51600930906FD93060900938705FDF2
:1063F00013860500E3E2FAFA93972900B38937017F
:106400009386160093991900B389B90083C50600D5
:10641000938909FD938705FD13860500E3FEFAFCC9
:106420006FF09FF70327C10083A7040083260700AE
:10643000130747002326E1002380D70003A40400AC
:106440001304140023A084006FF09FC5930710006D
:1064500063D4070F8327C1009386770093F686FFE6
:10646000938786002326F10083A9460083A70600B0
:1064700063DE090E83A604001306D002B307F040C2
:106480002380C60003A40400B336F000B3093041F2
:106490001304140023A08400138B0700B389D94090
:1064A000930CA000232401006FF05FCE03C61600FA
:1064B00013081800930609006FF0DFC383A70400D8
:1064C000138908006FF09FE9E3729BCF93071000D8
:1064D000930B000093061000E3C447D36FF05FD422
:1064E00097AC0100938C8CF59385090013850C0003
:1064F000EF109009330AAA406352400303A404003A
:106500002300A40103A40400130AFAFF13041400D7
:1065100023A08400E3160AFE130A000083C70C00C0
:10652000E38207E0E3CC09DA9389F9FF1307F0FF70
:10653000E396E9DA6FF0DFDC8327C100938647003A
:1065400083A707002326D10093D9F7416FF05FF2AC
:10655000635640019307D002E314FDF897AC0100A5
:10656000938CCCED930780026FF01FD7138B07003D
:10657000930CA0002324010003A404006FF01FC1AA
:10658000130101EB232E3113B70900409387F9FF64
:106590002324811423229114232C4113232A5113E1
:1065A0002326111423202115232861132326711378
:1065B00023248113232291132320A113232EB1110D
:1065C000130A05002324B10017A4010013040406D4
:1065D000973A0300938A0A2B97A40100938404B886
:1065E0002326F100930550021305A00013080004B0
:1065F000B70610F083470A00638EB7046388070A62
:1066000003270400130A1A00130617003387EA0051
:1066100097A8010023ACC8002300F7006380A708F7
:10662000E31A06FD173703001307C72513071700E2
:106630008347F7FF23A0F6F0832704009387F7FF33
:1066400017A601002324F6FEE39207FE83470A0003
:10665000E396B7FA83461A0013051A0013070500DC
:10666000930B0002130BF0FF130CF0FF1308000054
:1066700093055005930890009387D6FD93F7F70F85
:10668000130A170063ECF54493972700B38797002C
:1066900083A70700B38797006780070017370300B9
:1066A0001307471EE31406F86FF0DFF48320C114CC
:1066B0000324811483244114032901148329C11361
:1066C000032A8113832A4113032B0113832BC11245
:1066D000032C8112832C4112032D0112832DC11131
:1066E0001301011567800000930C8000130D00005A
:1066F0009307100063DA07218327810093877700CF
:1067000093F787FF83AD070003AB4700138787002C
:106710002324E10013860C009306000013850D006E
:1067200093050B00EF20C01B2328A10063086D45D3
:10673000130941019309100013860C009306000011
:1067400013850D0093050B00EF10D03B13860C0052
:1067500093060000930D0500138B0500EF204018F1
:106760002320A9009389190013094900E3166DFD40
:10677000E3F49DFD13060004B70610F063D489030B
:106780008327040013871700B387FA0097A5010039
:1067900023AEE5E823807701630AC706130CFCFFEC
:1067A000E3C089FF8327C1001305C100930890004F
:1067B000B386F9009396260093070101B386D700AC
:1067C0001308A00013030004370610F0E38CA6E0C2
:1067D00083A706009305000363F4F8009305700592
:1067E00003270400B387B700930517003387EA0037
:1067F00017AE0100232CBEE22300F70063860737A3
:10680000638C65329386C6FF6FF05FFC1737030019
:1068100013074707130717008347F7FF23A0F6F076
:10682000832704009387F7FF97A5010023A0F5E0D5
:10683000E39207FE130CFCFF6FF09FF68327040022
:10684000130600041387170097A5010023A0E5DEB7
:10685000B386FA00930500032380B6006308C7508F
:106860009387270097A6010023A2F6DC3387EA006E
:10687000930680072300D70017370300130787000C
:10688000B70610F06392C702130717008347F7FF9C
:1068900023A0F6F0832704009387F7FF17A60100D3
:1068A0002326F6D8E39207FE83278100930C00018C
:1068B000130D00009387470003278100130B00008E
:1068C000832D07002324F1006FF0DFE4832781008C
:1068D00083AC070013894700638E0C4C6358802BF0
:1068E0009307D0026394FB3E03C70C009305070097
:1068F0006314072A6F00002F93071000930CA00069
:10690000130D0000E3CA07DF832781009387470048
:106910006FF09FFA832781008346170013070A0050
:1069200003AB0700938747002324F100E3560CD400
:10693000130C0B00130BF0FF6FF01FD483461700EE
:10694000930BD00213070A006FF01FD39347FCFF8D
:1069500093D7F74183461700337CFC0013070A00E6
:106960006FF09FD183461700930B000313070A00B3
:106970006FF09FD003461700138B06FD13070A0024
:10698000930706FD93060600E3E2F8FA93172B003F
:10699000B38767011307170093971700B387C700E2
:1069A00003460700138B07FD930706FD93060600B9
:1069B000E3FEF8FC6FF09FF7832581008327040036
:1069C0001306A00003A7050093861700B387FA00FB
:1069D00017A50100232CD5C42380E70013894500A7
:1069E0006300C736930700046384F62A2324210139
:1069F0006FF05FBF9307100063DE073583278100C8
:106A000013877700137787FF930787002324F1000C
:106A1000032B47008327070063560B3E0327040020
:106A2000130600049306170097A5010023A0D5C004
:106A30003387EA009305D0022300B700638CC63881
:106A4000B307F0403337F000330B6041938D0700FC
:106A5000330BEB40930CA000130D00006FF09FCBA5
:106A6000834617001308180013070A006FF0DFC0F1
:106A70008346170013070A006FF01FC08327040026
:106A8000930600041387170017A601002320E6BA17
:106A9000B387FA00130650022380C700E314D7B46B
:106AA00017370300130707DEB70610F013071700A8
:106AB0008347F7FF23A0F6F0832704009387F7FFAF
:106AC00017A601002324F6B6E39207FE6FF09FB1EC
:106AD000930C0001130D00006FF09FC18327040089
:106AE00093060004130A05001387170017A6010078
:106AF000232EE6B2B387FA00130650022380C700A4
:106B0000E312D7AE173703001307C7D7B70610F045
:106B1000130717008347F7FF23A0F6F0832704002D
:106B20009387F7FF17A601002322F6B0E39207FE32
:106B3000130A05006FF01FAB17370300130787D444
:106B4000130717008347F7FF2320F6F0832704007D
:106B50009387F7FF97A5010023AAF5ACE39207FE00
:106B60009386C6FF6FF09FC617370300130787D1C0
:106B7000E39805FC9386C6FF6FF05FC5E3FA9DBB03
:106B8000930910006FF01FBF130C000003C70C0027
:106B900093050700E30C07E49308F0FF1305A0003A
:106BA00013080004B70610F0635E0B0C8327040083
:106BB00013861700B387FA0017A301002328C3A682
:106BC0002380E7006382A5086308060B938C1C00F2
:106BD00003C70C00130CFCFF93050700E31607FC2A
:106BE000E35680E1832704009305000213060004A6
:106BF000B70610F06F00C000130CFCFFE3080CDEBA
:106C000013871700B387FA002380B70017A5010088
:106C1000232EE5A093070700E310C7FE17370300F4
:106C2000130747C6130717008347F7FF23A0F6F0A3
:106C3000832704009387F7FF17A501002328F59EFB
:106C4000E39207FE6FF05FFB17370300130787C35C
:106C5000E30E06F6130717008347F7FF23A0F6F0AD
:106C6000832704009387F7FF17A601002320F69CD3
:106C7000E39207FE6FF09FF517370300130787C0F5
:106C80006FF05FFD130BFBFFE3121BF36FF05FF57B
:106C900017370300130707BFB70610F013071700D5
:106CA0008347F7FF23A0F6F0832704009387F7FFBD
:106CB00017A60100232CF696E39207FE2324210158
:106CC0006FF05F92979C0100938C4C7793050B00BB
:106CD00013850C00EF10400B330CAC40E35880EBF5
:106CE0008327040013060004B70610F06F00C000ED
:106CF000130CFCFFE30A0CE813871700B387FA00B4
:106D00002380770197A5010023A2E592930707004E
:106D1000E310C7FE173703001307C7B613071700A2
:106D20008347F7FF23A0F6F0832704009387F7FF3C
:106D300097A5010023ACF58EE39207FE6FF05FFB91
:106D400017370300130707B4E39806F4232421013F
:106D50006FF05F89832781001387470083A70700AF
:106D60002324E10013DBF7416FF01FCB173703003B
:106D7000130747B1B70610F0130717008347F7FF53
:106D800023A0F6F0832704009387F7FF17A60100DE
:106D9000232EF688E39207FE9307100017A7010041
:106DA0002326F7889307800717370300230CF7ACD7
:106DB0006FF09FAF635680019307D002E394FBF01E
:106DC000979C0100938C8C671307800293058002C7
:106DD0006FF09FDC973603009386C6AA370610F043
:106DE0009386160003C7F6FF2320E6F0032704006E
:106DF0001307F7FF97A5010023AAE582E31207FE18
:106E00006FF01FC4938D0700930CA000130D0000BA
:106E10006FF05F90B70710F023A0A7F26F0000009B
:106E2000130101FC130341022322B1029305030065
:106E3000232E11002324C1022326D1022328E1029C
:106E4000232AF102232C0103232E110323266100A0
:106E5000EFF00FF38320C1011305000013010104BB
:106E600067800000130101FB1303810323248102C7
:106E70002326A100232CC1021304050013060300DE
:106E80001305C100232611022322F104232ED1026F
:106E90002320E1042324010523261105232E61006C
:106EA000EFF04F9B8327C100238007000325C1001B
:106EB0008320C102330585400324810213010105AB
:106EC00067800000B70710F083A647F403A607F415
:106ED00003A747F4E31AD7FEB7160000938606FA15
:106EE000B306D60033B6C600B305E60023A4D7F434
:106EF00023A6B7F467800000B70710F003A747F494
:106F000003A607F483A647F4E31AD7FEB7160000DA
:106F1000938606FAB306D60033B6C60023A4D7F488
:106F2000B305E60023A6B7F49307000873A0473023
:106F300067800000130101FF232481002326110034
:106F4000979701009387076F179401001304446E0D
:106F500003A70700832704001306F07C9306470667
:106F6000938747069795010023A6D56C9795010056
:106F700023A0F56C634AD6008320C100032481005E
:106F800013010101678000001307478997970100EB
:106F900023A2E76AEF009047930710006316F502FB
:106FA00003270400B71700009387F7761305000046
:106FB000E3D4E7FCEFF01FE6032481008320C10047
:106FC000130101016FB05FB71795010013058547E5
:106FD000EFF01FE513052000EFF0DFE3032481004D
:106FE0008320C100130101016FB01FB51795010087
:106FF000130505476FF0DFE2179501001305C5463D
:107000006FF01FE2130101FF23248100232291006E
:1070100023261100B71400001794010013044445FF
:1070200093878438130000009387F7FFE39C07FEE3
:1070300013050400EFF0DFDE6FF09FFE1305000084
:107040006F001023130101FF23261100EF00103CF5
:107050001307100093070000631AE5008320C100A6
:1070600013850700130101016780000017950100D7
:107070001305453DEFF0DFDA8320C10093072000C0
:10708000138507001301010167800000737004304D
:107090006F00000067800000737004306F00000014
:1070A000130101FB9797010093870759232E3103A2
:1070B00083A907009797010093874758232021054C
:1070C00003A907009797010093878757232291040C
:1070D00083A407002326310123282101232A9100BC
:1070E0008327C10083250101232481040324410156
:1070F00023286103130B05001385070023261104C1
:10710000232C4103232A510323267103EF10504DF2
:1071100093050400EF200065232EA100930A0000D0
:10712000179A0100130A0A52B70B00802326310177
:1071300023282101232A91000325C1008325010171
:1071400003244101EF10D04993050400EF20806132
:10715000232CA100032581018325C101EF20901775
:1071600093050000EF20405363420504032581018D
:107170008325C101EF20101683250A00EF2000456A
:107180003325A00063100502E3920AFA83570B002F
:10719000938717009397070193D707012310FB00EC
:1071A0006FF0DFF8930A10006FF05FF8032581019C
:1071B0008325C10133C5AB00EF20D01183250A0020
:1071C000EF20C0403325A0006FF0DFFB130101FB6F
:1071D0009797010093874747232E310383A9070020
:1071E00097970100938787462320210503A907006D
:1071F000979701009387C7452322910483A4070032
:107200002326310123282101232A91008327C1004D
:1072100083250101232481040324410123286103E0
:10722000130B05001385070023261104232C4103AB
:10723000232A510323267103EF10D07F9305040006
:10724000EF204052232EA100930A0000179A01005C
:10725000130A4A3FB70B008023263101232821015E
:10726000232A91000325C100832501010324410144
:10727000EF10507C93050400EF20C04E232CA1009A
:10728000032581018325C101EF20D004930500006F
:10729000EF20804063420504032581018325C1015D
:1072A000EF20500383250A00EF2040323325A00051
:1072B00063100502E3920AFA83570B0093871700C5
:1072C0009397070193D707012310FB006FF0DFF8B6
:1072D000930A10006FF05FF8032581018325C10137
:1072E00033C5AB00EF20007F83250A00EF20002E7E
:1072F0003325A0006FF0DFFB130101FA2326A10064
:1073000013058002232C8104232A910423263105AE
:10731000232441052322510523206105232E7103D7
:10732000232C8103232A91032328A1032326B103BD
:10733000232E110423282105EFE08FF497970100F5
:107340009387473183A40700130405002324010019
:10735000938D0400138D0400938C0400138C04009F
:10736000938B0400138B0400938A0400138A040097
:1073700093890400930700002328F100232AF100D9
:10738000232EF1000325C10193850400EF20803DE9
:107390002320A4000325C1010329010193850D00C9
:1073A000EF20403C93050900EF1090232328A10013
:1073B0000325C10193050D00EF20C03A2322A4004C
:1073C0000325C1010329010193850C00EF208039B9
:1073D00093050900EF10D0202328A1000325C10147
:1073E00093050C00EF2000382324A4000325C101DD
:1073F0000329010193850B00EF20C0369305090096
:10740000EF10101E2328A1000325C10193050B00D6
:10741000EF2040352326A4000325C10103290101E3
:1074200093850A00EF20003493050900EF10501BEC
:107430002328A1000325C10193050A00EF20803213
:107440002328A4000325C101032901019385090014
:10745000EF20403193050900EF1090189797010035
:107460009387471F2328A1000325C10183A5070097
:10747000EF20402F979701009387C71D232AA40070
:107480000325C10183A5070003290101EF20802DF9
:1074900093050900EF10D014979701009387871B7D
:1074A0002328A1000325C10183A50700EF20802B1D
:1074B000979701009387071A232CA4000325C10185
:1074C00083A5070003290101EF20C02993050900C6
:1074D000EF101011979701009387C7172328A10079
:1074E0000325C10183A50700EF20C027979701005E
:1074F00093874716232EA4000325C10183A5070007
:1075000003290101EF20002693050900EF10500D1B
:1075100097970100938707142328A1000325C10131
:1075200083A50700EF200024979701009387871217
:107530002320A40283A507000325C101032901011B
:10754000EF20402293050900EF1090099797010062
:10755000938747102328A1000325C10183A50700B5
:10756000EF204020979701009387C70E2322A402A3
:107570000325C10183A5070003290101EF20801E17
:1075800093050900EF10D0052328A100032504006E
:1075900083254101EF10D004232AA10003254400D4
:1075A00083254101EF10D003232AA1000325840085
:1075B00083254101EF10D002232AA1000325C40036
:1075C00083254101EF10D001232AA10003250401E6
:1075D00083254101EF10D000232AA1000325440197
:1075E00083254101EF10C07F232AA10003258401D8
:1075F00083254101EF10C07E232AA1000325C40189
:1076000083254101EF10C07D232AA1000325040238
:1076100083254101EF10C07C232AA10003254402E9
:1076200083254101EF10C07B232AA100032501011E
:1076300083254101EF20004A232CA100032581016D
:1076400093050000EF20400563480504979701006B
:10765000938747FF0325810183A50700EF1010776B
:107660003325A0006314050283278100E39407D02B
:107670000327C100835707009387170093970701DB
:1076800093D707012310F7006FF0DFCE93071000A8
:107690002324F1006FF01FCE979701009387C7FB5B
:1076A0000325810183A50700EF10107F1355F50115
:1076B0006FF05FFB130101FA2326A100130580027E
:1076C000232C8104232A91042326310523244105F8
:1076D0002322510523206105232E7103232C8103CE
:1076E000232A91032328A1032326B103232E110467
:1076F00023282105EFE0CFB897970100938707F67D
:1077000083A407001304050023240100938D0400C3
:10771000138D0400938C0400138C0400938B0400DD
:10772000138B0400938A0400138A040093890400D5
:10773000930700002328F100232AF100232EF100F3
:107740000325C10193850400EF1080692320A40064
:107750000325C1010329010193850D00EF10406845
:1077600093050900EF10C0672328A1000325C1017C
:1077700093050D00EF10C0662322A4000325C1016C
:107780000329010193850C00EF1080659305090022
:10779000EF1000652328A1000325C10193050C000B
:1077A000EF1000642324A4000325C1010329010173
:1077B00093850B00EF10C06293050900EF10406243
:1077C0002328A1000325C10193050B00EF104061A0
:1077D0002326A4000325C1010329010193850A0082
:1077E000EF10006093050900EF10805F2328A100CF
:1077F0000325C10193050A00EF10805E2328A40031
:107800000325C1010329010193850900EF10405DA3
:1078100093050900EF10C05C97970100938707E478
:107820002328A1000325C10183A50700EF10405BB9
:1078300097970100938787E2232AA4000325C101BB
:1078400083A5070003290101EF1080599305090062
:10785000EF10005997970100938747E02328A10074
:107860000325C10183A50700EF10805797970100FA
:107870009387C7DE232CA4000325C10183A507003D
:1078800003290101EF10C05593050900EF10405581
:1078900097970100938787DC2328A1000325C10166
:1078A00083A50700EF10C05397970100938707DB6C
:1078B000232EA4000325C10183A50700032901018C
:1078C000EF10005293050900EF10805197970100C7
:1078D0009387C7D82328A1000325C10183A50700EA
:1078E000EF10005097970100938747D72320A402F9
:1078F00083A507000325C10103290101EF10404EB4
:1079000093050900EF10C04D97970100938707D5A5
:107910002328A1000325C10183A50700EF10404CD7
:1079200097970100938787D32322A4020325C101DF
:1079300083A5070003290101EF10804A9305090080
:10794000EF10004A2328A1000325040083254101EC
:10795000EF100049232AA10003254400832541019B
:10796000EF100048232AA10003258400832541014C
:10797000EF100047232AA1000325C40083254101FD
:10798000EF100046232AA1000325040183254101AD
:10799000EF100045232AA10003254401832541015E
:1079A000EF100044232AA10003258401832541010F
:1079B000EF100043232AA1000325C40183254101C0
:1079C000EF100042232AA100032504028325410170
:1079D000EF100041232AA100032544028325410121
:1079E000EF100040232AA100032501018325410156
:1079F000EF20400E232CA1000325810193050000F8
:107A0000EF1090496348050497970100938787C357
:107A10000325810183A50700EF10503B3325A0000B
:107A20006314050283278100E39407D00327C10074
:107A300083570700938717009397070193D7070190
:107A40002310F7006FF0DFCE930710002324F1001E
:107A50006FF01FCE97970100938707C00325810120
:107A600083A50700EF1050431355F5016FF05FFB3E
:107A7000130101FF232481001307050013040500EF
:107A800093080000130800009307000097260300E6
:107A9000938646E313060040979501009385859EE3
:107AA00017F5FFFF1305056023261100EFA08F9D3A
:107AB0001307040093080000130800009307000058
:107AC00097260300938626E0130600409795010051
:107AD0009385C59B17F5FFFF1305856FEFA08F9A60
:107AE0001307040093080000130800009307000028
:107AF00097260300938646DD130600409795010004
:107B00009385459917050000130505BBEFA08F97D6
:107B100013070400930800001308000093070000F7
:107B200097260300938666DA1306004097950100B6
:107B30009385C59617F5FFFF1305457CEFA08F943D
:107B400013070400930800001308000093070000C7
:107B500097260300938686D7130600409795010069
:107B60009385459417F5FFFF1305C553EFA08F913B
:107B70001307040093080000130800009307000097
:107B8000972603009386A6D413060040979501001C
:107B90009385C59117F5FFFF13058563EFA08F8EC1
:107BA0001307040093080000130800009307000067
:107BB000972603009386C6D11306004097950100CF
:107BC0009385458F17050000130505AFEFA08F8B38
:107BD00013070400032481008320C10093080000E0
:107BE000130800009307000097260300938666CED3
:107BF00013060040979501009385458C17F5FFFF0C
:107C00001305C56F130101016FA0CF87172803006B
:107C1000035848CB172703000357E7CB172E030061
:107C2000035E4ECA9726030083D6E6C99727030052
:107C300083D747CA172303000353E3C8172503005C
:107C4000035585C917260300035606C83307D740D6
:107C50009728030083D848C79725030083D5E5C735
:107C60009726030083D666C6B38707413305C54010
:107C70003337E00017280300035828C517260300F0
:107C80000356C6C5972F030083DF4FC43307E04078
:107C9000B385D540B337F0003335A000972E0300ED
:107CA00083DECEC29726030083D666C3172F030058
:107CB000035FEFC1B3F7E7003305A0403306F64199
:107CC000B335B000972F030083DF6FC01727030081
:107CD000035707C19723030083D383BFB3F7A700DC
:107CE000B305B040B386E6413336C000172F03001A
:107CF000035F0FBE172503000355A5BE972203009F
:107D000083D222BDB3F7B7003306C04033077740B4
:107D1000B336D000B306D040B3F7C70033055540A3
:107D20003337E000B3F7D7003307E0403335A00026
:107D3000B3F7E7003305A04017270300035767B9DF
:107D4000972603002398C6B997260300239566B8A3
:107D500097260300239216B997260300239F06B7A0
:107D600097260300239CD6B7972603002399F6B7DE
:107D7000972603002396E6B7972603002393E6B6DB
:107D800033F5A70067800000B305B5009307050031
:107D90006386B70003C70700631607003385A74053
:107DA00067800000938717006FF09FFE130101FBAF
:107DB00023229104232C410323229103232611041F
:107DC0002324810423202105232E3103232A510358
:107DD0002328610323267103232481032320A10385
:107DE000232EB101930C0500138A050093040000B3
:107DF00063DE05003305A0403337A000B305B04073
:107E0000930C0500338AE5409304F0FF63DA060023
:107E10003306C040B337C000B306D040B386F64047
:107E2000930A06009389060013840C0013090A00C4
:107E300063960628178B0100130B4B4F6370CA160D
:107E4000B70701006372F6149307F00F63F4C700DD
:107E500093098000B3573601330BFB0083470B00B7
:107E600013050002B3873701B309F540638C09009D
:107E7000B3153A01B3D7FC00B31A360133E9B700A2
:107E800033943C0113DB0A0193050B001305090031
:107E9000EF200013130A050093050B00939B0A01C2
:107EA00013050900EF20400D93DB0B01930505003E
:107EB00013850B00EF208009131A0A019357040160
:107EC000B367FA0063FAA700B387570163E6570167
:107ED00063F4A700B38757013389A74093050B00CC
:107EE00013050900EF20C00D130A050093050B00D0
:107EF00013050900EF204008131404019305050041
:107F0000131A0A0113850B0013540401EF20000417
:107F100033648A00637AA400330454016366540115
:107F20006374A400330454013304A4403354340173
:107F300093050000638A040033048040B337800057
:107F4000B305B040B385F540130504008320C10498
:107F50000324810483244104032901048329C103E8
:107F6000032A8103832A4103032B0103832BC102CC
:107F7000032C8102832C4102032D0102832DC101B8
:107F80001301010567800000B70700019309000194
:107F9000E362F6EC930980016FF0DFEB631A0600F1
:107FA0009305000013051000EF10107D930A0500E3
:107FB000B707010063FAFA0E9307F00F63F4570155
:107FC00093098000B3D73A01330BFB0083470B00C2
:107FD0001305000233095A41B3873701B309F5404D
:107FE000E38209EAB39A3A01335BFA00B3153A0126
:107FF000B3D7FC0093DB0A0133E9B70013050B008C
:1080000093850B00EF10D07B130A050093850B00BE
:10801000139C0A0113050B00EF101076135C0C0182
:108020009305050013050C00EF105072131A0A0196
:1080300093570901B367FA0033943C0163FAA70030
:10804000B387570163E6570163F4A700B38757016D
:10805000338BA74093850B0013050B00EF10507670
:10806000130A050093850B0013050B00EF10D07069
:108070009305050013050C00EF10506D93160901D0
:10808000131A0A0193D60601B366DA0063FAA60052
:10809000B386560163E6560163F4A600B386560123
:1080A0003389A6406FF01FDEB70700019309000176
:1080B000E3EAFAF0930980016FF0DFF06376DA000B
:1080C00093050A006FF01FE7B707010063FAF60493
:1080D000930BF00F33B5DB001315350033D7A60033
:1080E0009787010093878724B387E70083CB070036
:1080F00093050002B38BAB00338B7541631C0B02FD
:1081000063E4460163EACC003384CC40B306DA4032
:1081100033B98C0033892641930509006FF09FE144
:10812000B707000113050001E3EAF6FA1305800121
:108130006FF0DFFAB3966601335D7601336DDD00D3
:10814000B35D7A01B3156A0133DC7C0113540D0170
:10815000336CBC0013850D0093050400B319660150
:10816000EF101066930A05009305040013850D00B7
:1081700033996C01931C0D01EF10106093DC0C011E
:10818000130A05009305050013850C00EF10105C21
:10819000939A0A0113570C0133E7EA00930D0A0082
:1081A000637EA7003307A701930DFAFF6368A70159
:1081B0006376A700930DEAFF3307A701330AA740B0
:1081C0009305040013050A00EF10905F9305040067
:1081D000930A050013050A00EF10105A93050500D5
:1081E0001304050013850C00EF10505693150C0175
:1081F000939A0A0193D50501B3E5BA001307040069
:1082000063FEA500B385A5011307F4FF63E8A5018C
:1082100063F6A5001307E4FFB385A501939D0D0147
:10822000B70C0100B3EDED001384FCFFB3F78D0034
:1082300033F48900338AA5401385070093050400B1
:108240002326F10093DD0D01EF105050930504003B
:10825000930A050013850D00EF10504F13DC090140
:1082600093050C002324A10013850D00EF10104E80
:108270008327C10013040C0093050400130C0500B0
:1082800013850700EF10904C8326810013D70A0155
:108290003305D5003307A7006374D700330C9C0166
:1082A000B70701009387F7FF935507013377F7006E
:1082B00013170701B3F7FA00B3858501B307F70079
:1082C0006366BA00631EBA00637CF90033863741E7
:1082D000B3B7C700B385A541B385F5409307060042
:1082E000B307F9403339F900B305BA40B3852541E6
:1082F00033947501B3D767013364F400B3D56501D6
:108300006FF05FC3130101FD23229102232A510163
:10831000232611022324810223202103232E31014D
:10832000232C41012328610123267101232481018B
:10833000232291012320A101930A050093840500C3
:10834000639E06381304060093090500178901008F
:108350001309C9FD63F8C512B7070100138B0500A7
:108360006378F6101307F00F3337C7001317370081
:10837000B357E6003309F900834609003387E60066
:1083800093060002B386E640638C0600B394D400E3
:1083900033D7EA003314D600336B9700B399DA0071
:1083A000935A040193850A0013050B00EF10504106
:1083B0001309050093850A00931B040113050B00A4
:1083C000EF10903B93DB0B01930405009305050030
:1083D00013850B00EF1090371319090193D709018A
:1083E000B367F900138A040063FEA700B387870010
:1083F000138AF4FF63E8870063F6A700138AE4FF9B
:10840000B3878700B384A74093850A0013850400CF
:10841000EF10103B1309050093850A001385040033
:10842000EF10903593990901930405009305050019
:108430001319090113850B0093D90901EF101031AD
:10844000B36939011386040063FCA900B309340140
:108450001386F4FF63E6890063F4A9001386E4FF42
:1084600013140A013364C400130A00006F000013E0
:10847000B707000113070001E36CF6EE1307800154
:108480006FF01FEF138A0600631A060093050000C1
:1084900013051000EF10502E13040500B70701005C
:1084A000637EF4129307F00F63F48700130A8000D1
:1084B000B35744013309F90003470900930600024A
:1084C00033074701B386E64063940612B3848440C1
:1084D000130A1000135B040193050B0013850400BD
:1084E000EF10102E1309050093050B0013850400EF
:1084F000931B0401EF10502893DB0B01930405003C
:108500009305050013850B00EF1050241319090182
:1085100093D70901B367F900938A040063FEA700AB
:10852000B3878700938AF4FF63E8870063F6A700A8
:10853000938AE4FFB3878700B384A74093050B00B9
:1085400013850400EF10D0271309050093050B00D5
:1085500013850400EF10502293990901930405003C
:10856000930505001319090113850B0093D909011F
:10857000EF10D01DB36939011386040063FCA90014
:10858000B30934011386F4FF63E6890063F4A9009C
:108590001386E4FF13940A013364C4001305040036
:1085A00093050A008320C10203248102832441022F
:1085B000032901028329C101032A8101832A410180
:1085C000032B0101832BC100032C8100832C41006C
:1085D000032D01001301010367800000B7070001AC
:1085E000130A0001E366F4EC130A80016FF05FECFC
:1085F0003314D40033DAE400B399DA0033D7EA0055
:10860000935A0401B394D40093850A0013050A0019
:10861000336B9700EF10D01A1309050093850A00F9
:1086200013050A00931B0401EF10101593DB0B01D7
:10863000930405009305050013850B00EF1010113E
:108640001319090113570B013367E900138A04005A
:10865000637EA70033078700138AF4FF63688700EF
:108660006376A700138AE4FF33078700B304A740AB
:1086700093850A0013850400EF1090141309050078
:1086800093850A0013850400EF10100F9304050072
:108690009305050013850B00EF10500B13170B010A
:1086A0001357070113190901B367E9001387040081
:1086B00063FEA700B38787001387F4FF63E8870092
:1086C00063F6A7001387E4FFB3878700131A0A0134
:1086D000B384A740336AEA006FF0DFDF63ECD51E96
:1086E000B707010063F4F6041307F00FB335D700A2
:1086F0009395350033D7B60097870100938707C35A
:10870000B387E70003C70700130A00023307B70067
:10871000330AEA4063160A0213041000E3E096E805
:1087200033B6CA00134416006FF05FE7B7070001C5
:1087300093050001E3E0F6FC930580016FF09FFBD9
:10874000B35CE600B3964601B3ECDC0033D4E4003E
:1087500093DB0C01B397440133D7EA0093850B00F8
:1087600013050400336BF700B3194601EF105005F1
:108770001309050093850B0013050400139C0C01DD
:10878000EF10807F135C0C01930405009305050036
:1087900013050C00EF10807B1319090113570B010F
:1087A0003367E90013840400637EA7003307970151
:1087B0001384F4FF636897016376A7001384E4FFD2
:1087C00033079701B304A74093850B00138504007A
:1087D000EF10007F1309050093850B00138504003B
:1087E000EF108079930405009305050013050C0034
:1087F000EF10C07593170B011319090193D70701E7
:10880000B367F9001386040063FEA700B3879701DE
:108810001386F4FF63E8970163F6A7001386E4FF6D
:10882000B387970113140401B70B01003364C4002C
:108830001389FBFF337D240133F92901B384A74059
:108840009305090013050D00EF104070935C0401BF
:1088500093050900130B050013850C00EF10006F42
:1088600093D90901130C05009385090013850C00A9
:10887000EF10C06D130905009385090013050D0065
:10888000EF10C06C3305850193570B013385A700AA
:10889000637485013309790193570501B387270173
:1088A00063E6F402E392F4BCB70701009387F7FF95
:1088B0003375F50013150501337BFB0033964A0130
:1088C00033056501130A0000E37AA6CC1304F4FF14
:1088D0006FF09FB9130A0000130400006FF01FCC63
:1088E000130101FB2324810423229104232E31034D
:1088F000232291032326110423202105232C410345
:10890000232A51032328610323267103232481038F
:108910002320A103232EB101930C050093890500A8
:108920001304050093840500639E062613090600C0
:10893000138A0600978A0100938A4A9F63F4C5143C
:10894000B70701006376F6129307F00F63F4C700D0
:10895000130A8000B3574601B38AFA0003C70A001E
:108960001305000233074701330AE540630C0A0090
:10897000B395490133D7EC0033194601B364B7000E
:1089800033944C01935A090193850A00138504001E
:10899000EF1000639309050093850A00131B09017A
:1089A00013850400EF10405D135B0B019305050078
:1089B00013050B00EF108059939909019357040197
:1089C000B3E7F90063FAA700B387270163E627013D
:1089D00063F4A700B3872701B384A74093850A00F7
:1089E00013850400EF10C05D9309050093850A000C
:1089F00013850400EF10405813140401930505007B
:108A00009399090113050B0013540401EF1000544E
:108A100033E48900637AA4003304240163662401EB
:108A20006374A400330424013304A4403355440187
:108A3000930500008320C10403248104832441049E
:108A4000032901048329C103032A8103832A4103E3
:108A5000032B0103832BC102032C8102832C4102CF
:108A6000032D0102832DC101130101056780000060
:108A7000B7070001130A0001E36EF6EC130A800148
:108A80006FF05FED631A06009305000013051000F8
:108A9000EF10804E13090500B7070100637AF90E45
:108AA0009307F00F63F42701130A8000B3574901BD
:108AB000B38AFA0003C70A0013050002B3842941F0
:108AC00033074701330AE540E30E0AEA3319490147
:108AD000B3DAE900B395490133D7EC0093540901A7
:108AE000336BB70013850A0093850400EF10404DE7
:108AF0009309050093850400931B090113850A005F
:108B0000EF10804793DB0B019305050013850B00E5
:108B1000EF10C0439399090193570B01B3E7F90094
:108B200033944C0163FAA700B387270163E627015A
:108B300063F4A700B3872701B38AA7409385040095
:108B400013850A00EF10C0479309050093850400C0
:108B500013850A00EF1040429305050013850B00B2
:108B6000EF10C03E93150B019399090193D50501B0
:108B7000B3E5B90063FAA500B385250163E62501D5
:108B800063F4A500B3852501B384A5406FF09FDF92
:108B9000B7070001130A0001E36AF9F0130A800124
:108BA0006FF0DFF0E3E8D5E8B707010063FCF604F7
:108BB000930BF00F33B5DB001315350033D7A60048
:108BC0009777010093878776B387E70083CB070009
:108BD00093050002B38BAB00338B7541631E0B0210
:108BE00063E4360163EACC003384CC40B386D940D9
:108BF00033B58C00B384A6401305040093850400AC
:108C00006FF05FE3B707000113050001E3E8F6FA30
:108C1000130580016FF09FFAB3966601335D76010C
:108C2000336DDD0033D47901B395690133DC7C0108
:108C300093540D01336CBC001305040093850400AC
:108C4000B31A6601EF10C037130A050093850400BC
:108C50001305040033996C01931C0D01EF10C03112
:108C600093DC0C01130405009305050013850C002B
:108C7000EF10C02D131A0A0113570C013367EA00D5
:108C8000130A0400637EA7003307A701130AF4FF49
:108C90006368A7016376A700130AE4FF3307A701FF
:108CA000B309A7409385040013850900EF104031F4
:108CB000938504001304050013850900EF10C02BF1
:108CC000930505009304050013850C00EF100028A0
:108CD00093150C011314040193D50501B365B40079
:108CE0001387040063FEA500B385A5011387F4FF75
:108CF00063E8A50163F6A5001387E4FFB385A5012A
:108D0000131A0A01B70C0100336AEA001384FCFF4E
:108D1000B3778A0033F48A00B384A5401385070033
:108D2000930504002326F100135A0A01EF100022D4
:108D3000930905009305040013050A00EF100021B4
:108D400013DC0A01930D050093050C0013050A00BE
:108D5000EF10C01F8327C100130A050093050C0004
:108D600013850700EF10801E3305B50113D70901E5
:108D70003307A7006374B701330A9A01B7070100EC
:108D80009387F7FF935507013377F7001317070110
:108D9000B3F7F900B3854501B307F70063E6B40004
:108DA000639EB400637CF90033865741B3B7C700B4
:108DB000B385A541B385F54093070600B307F94095
:108DC0003339F900B385B440B38525413394750137
:108DD000B3D767013365F400B3D565016FF09FC564
:108DE000B7078000130101FF9387F7FF33F7A70050
:108DF0002324810023202101135475011359F50107
:108E000013D57501B3F7B7001374F40F1375F50F8D
:108E1000232611002322910093D5F5011316370064
:108E2000939737003307A440631EB9186358E00ACC
:108E300063180506639C07009307F00F630CF404A6
:108E400093070600130504006F00C00B1307F7FF1C
:108E5000631E0702B387C70013050400139757006A
:108E60006352070A130515001307F00F6304E53278
:108E70003707007E93F617001307F7FF93D7170005
:108E8000B3F7E700B3E7D7006F00C0079306F00F12
:108E90006310D402930706001305F00F6F008006DD
:108EA0009306F00FE308D4FEB7060004B3E7D7003B
:108EB0009306B00163D6E600930710006FF09FF9A8
:108EC00093060002B386E640B3D5E700B397D70018
:108ED000B337F000B3E7F5006FF0DFF7630407087E
:108EE00063100404630006029306F0FF6316D700C4
:108EF000B387C7006FF09FF69306F00F1347F7FF95
:108F0000631AD50213F777006308072813F7F700F1
:108F1000930640006302D728938747006F00C0275D
:108F20009306F00FE300D5FEB70600043307E040D8
:108F30003366D6009306B00163D6E600130710002F
:108F40006F00C00193060002B355E6003387E64088
:108F50003317E6003337E00033E7E500B387E70077
:108F60006FF0DFEF130514009376F50F1307100071
:108F70006340D7046318040213050000E30406F8F5
:108F800063860720B387C70013975700E35C07F693
:108F9000370700FC1307F7FFB3F7E70013051000CE
:108FA0006FF05FF6E30A06EE639407166FF09FEE2C
:108FB0001307F00F6300E51E3307F6009357170001
:108FC0006FF05FF46350E00863160504E38607E67C
:108FD0001307F7FF63140702B307F64013050400F5
:108FE00013975700E35007F2B70400049384F4FF8B
:108FF000B3F49700130405006F00C0139306F00F3D
:10900000E30AD4E89306B00163D0E60293071000A8
:109010006FF09FFC9306F00FE30ED4E6B706000452
:10902000B3E7D7006FF01FFE93060002B3D5E70049
:109030003387E640B397E700B337F000B3E7F500B6
:109040006FF09FF9630E0706631E04021389050083
:10905000E30A06EA9306F0FF6318D700B387C74018
:10906000138905006FF0DFF79306F00F1347F7FF42
:10907000E30AD5E89306B00163D4E60213071000B3
:109080006F0080039306F00F13890500E30CD5E60B
:10909000B70600043307E0403366D6006FF09FFD4B
:1090A000930600023358E6003387E6403317E600A4
:1090B0003337E0003367E800B387E7406FF05FFACB
:1090C000130714001377F70F9306100063CAE60422
:1090D000631C040263180600639E07121305000058
:1090E0006F008003638C07123307F6409316570016
:1090F000B387C74063C006129307070063160706CD
:10910000930700006FF09FFDE31006EA639C0710D1
:10911000B70700021305F00F130900006F00C00726
:10912000B304F6401397540063540704B384C74054
:109130001389050013850400EF00D06E1305B5FFF9
:10914000B394A400634A85023305854013051500D6
:1091500013040002B3D7A4003305A440B394A400C1
:10916000B3349000B3E79700130500006FF09FD968
:10917000E38804F86FF01FFCB70700FC9387F7FF44
:109180003305A440B3F7F4006FF0DFD79307060070
:109190006FF05FD79307000013975700635E0700D7
:1091A000130515001307F00F6302E508370700FCED
:1091B0001307F7FFB3F7E7001307F00F93D7370054
:1091C0006318E50063860700B70740001309000035
:1091D000370780001307F7FF1375F50FB3F7E700A4
:1091E00013177501370580808320C1000324810097
:1091F0001305F5FF33F5A7001319F9013365E500F1
:109200003365250183244100032901001301010175
:1092100067800000138905006FF01FF593070600B3
:109220006FF09FF4138905006FF01FC793070000CC
:109230006FF09FF8130101FD23229102232A5101AF
:1092400093547501B70A800023202103232861016C
:10925000938AFAFF2326110223248102232E31014F
:10926000232C4101232671012324810193F4F40F5F
:10927000138B0500B3FAAA001359F501638804089B
:109280009307F00F6384F40A939A3A00B707000437
:10929000B3EAFA00938414F8930B000013557B0192
:1092A000370480001304F4FF1375F50F3374640161
:1092B000135BFB01630C05089307F00F6308F50AC5
:1092C00013143400B70700043364F400130515F8D1
:1092D0009307000013972B003367F7001307F7FF7E
:1092E0009306E000B3496901338AA44063E0E60ACB
:1092F00097760100938606FC131727003307D700E3
:10930000032707003307D70067000700638A0A02B4
:1093100013850A00EF0010519307B5FF9304A0F8DE
:10932000B39AFA00B384A4406FF01FF79304F00FD0
:10933000930B2000E3840AF6930B30006FF01FF6C6
:1093400093040000930B10006FF05FF5630A0402B2
:1093500013050400EF00104D9307B5FF3314F4001C
:109360009307A0F83385A7406FF09FF61305F00F21
:1093700093072000E30004F6930730006FF09FF599
:1093800013050000930710006FF0DFF4131B540067
:1093900063F68A12130AFAFF13090000935B0B01AC
:1093A0003704010093850B001304F4FF13850A00B2
:1093B000EF00903C33748B0093050500130C0500FF
:1093C00013050400EF0090389304050093850B000B
:1093D00013850A00EF00D03E13590901131505014A
:1093E0003365A90013090C00637E95003305650100
:1093F0001309FCFF63686501637695001309ECFFB0
:1094000033056501B304954093850B001385040073
:10941000EF00903693050500130C050013050400BA
:10942000EF00D032930A050093850B0013850400EA
:10943000EF0010391315050113040C00637E55016C
:10944000330565011304FCFF63686501637655010C
:109450001304ECFF33056501131909013305554168
:10946000336989003335A0003364A9001307FA0774
:109470006350E00A93777400638A07009377F400DF
:10948000930640006384D7001304440093174400FC
:1094900063DA0700B70700F89387F7FF3374F40027
:1094A00013070A089307E00F1354340063D2E70C44
:1094B000130400001307F00F6F00800B1399FA01DB
:1094C00093DA1A006FF09FED9309090013840A00E4
:1094D00093870B0013072000E38CE7FC1307300091
:1094E0006382E70813071000E392E7F81304000013
:1094F000130700006F00C00793090B006FF09FFD7A
:109500003704400093090000930730006FF09FFC80
:1095100093071000B387E7401307B001E348F7FC57
:109520001305EA09B357F4003314A4003334800060
:1095300033E4870093777400638A07009377F4001D
:10954000130740006384E70013044400931754009A
:1095500013543400E3DE07F813040000130710006F
:109560006F000001370440001307F00F930900005B
:10957000370580001305F5FF3374A400370580809C
:109580001305F5FF1377F70F3374A4001317770152
:109590001395F9013364E4003365A4008320C1020C
:1095A0000324810283244102032901028329C1018A
:1095B000032A8101832A4101032B0101832BC1006E
:1095C000032C81001301010367800000370780002E
:1095D0001307F7FF935675013378A70013D675016B
:1095E0009357F50193F6F60F1305F00F3377B70095
:1095F0001376F60F93D5F5016398A6001305E0FFE7
:10960000630E0806678000006318A6001305E0FFDC
:10961000630E070667800000639406061335180082
:109620006314060063060704631C05006394B70017
:10963000635ED60013051000639607006780000084
:10964000E39E05FE1305F0FF6780000063DAC600A5
:109650001305F0FFE38407FE130510006780000088
:10966000E36A07FD13050000E364E8FE6FF01FFDE9
:1096700013050000E30408FC6FF0DFFBE308D6F8F5
:10968000E31606FAE30807FA6FF05FFA13351800DD
:10969000E38C06F86FF09FF9370780001307F7FF98
:1096A000935675013378A70013D675019357F501CA
:1096B00093F6F60F1305F00F3377B7001376F60F16
:1096C00093D5F5016398A60013052000630E0806E4
:1096D000678000006318A60013052000630E0706CC
:1096E00067800000639406061335180063140600B3
:1096F00063060704631C05006394B700635ED6002D
:10970000130510006396070067800000E39E05FEC6
:109710001305F0FF6780000063DAC6001305F0FF51
:10972000E38407FE1305100067800000E36A07FD6D
:1097300013050000E364E8FE6FF01FFD1305000051
:10974000E30408FC6FF0DFFBE308D6F8E31606FA43
:10975000E30807FA6FF05FFA13351800E38C06F898
:109760006FF09FF9130101FD2322910223202103B1
:10977000B704800013597501232E3101232671018E
:109780009384F4FF2326110223248102232C410118
:10979000232A5101232861012324810123229101DD
:1097A0001379F90F938B0500B3F4A4009359F501D5
:1097B000630A09089307F00F6306F90A93943400CB
:1097C000B7070004B3E4F400130919F8130B000001
:1097D00013D57B01370480001304F4FF1375F50FD4
:1097E0003374740193DBFB01630E05089307F00FDC
:1097F000630AF50A13143400B70700043364F40055
:10980000130515F89306000093172B00B3E7D70054
:109810003309A9009387F7FF1307E00033CA7901E2
:10982000930A19006360F70A17770100130747AC22
:1098300093972700B387E70083A70700B387E70064
:1098400067800700638A040213850400EF00807DAF
:109850009307B5FF1309A0F8B394F4003309A940A6
:109860006FF0DFF61309F00F130B2000E38204F60C
:10987000130B30006FF0DFF513090000130B10001D
:109880006FF01FF5630A040213050400EF008079EE
:109890009307B5FF3314F4009307A0F83385A7406E
:1098A0006FF05FF61305F00F93062000E30E04F44B
:1098B000930630006FF05FF513050000930610006B
:1098C0006FF09FF4370C0100130BFCFF93DB0401D6
:1098D000935C0401B3F464013374640193050400E0
:1098E00013850400EF0080669305040093090500CA
:1098F00013850B00EF0080651304050093850C00B1
:1099000013850B00EF008064930B05009385040022
:1099100013850C00EF0080633305850093D70901A0
:109920003385A70063748500B38B8B01B377650122
:1099300093970701B3F96901B3873701139467005F
:109940003334800093D7A70113550501B367F400A2
:1099500033047501131464003364F4009317440056
:1099600063D6070E935714001374140033E4870072
:109970001387FA076350E00E93777400638A070039
:109980009377F400930640006384D70013044400E7
:109990009317440063DA0700B70700F89387F7FFCF
:1099A0003374F40013870A089307E00F63C4E710C9
:1099B000935734006F000003138A090013840400D6
:1099C00093060B00930720006386F60E9307300082
:1099D000638AF60C130610009307000013070000BB
:1099E000E398C6F8370480001304F4FF370580803D
:1099F000B3F787001305F5FF8320C102032481021A
:109A00001377F70FB3F7A700131777011315FA01B0
:109A1000B3E7E70083244102032901028329C1013E
:109A2000032A8101832A4101032B0101832BC100F9
:109A3000032C8100832C410033E5A70013010103AF
:109A400067800000138A0B006FF0DFF7930A0900AC
:109A50006FF01FF293071000B387E7401307B001C0
:109A60006340F706938AEA09B357F40033145401AC
:109A70003334800033E4870093777400638A0700EF
:109A80009377F400130740006384E7001304440055
:109A90009317540063CA070293573400130700005A
:109AA0006FF05FF4B70740001307F00F130A0000D0
:109AB0006FF05FF3930700001307F00F6FF09FF252
:109AC000930700006FF09FFD93070000130710003D
:109AD0006FF05FF1B70780009387F7FF130101FF75
:109AE00033F7A7009356750113D67501B3F7B70086
:109AF000232291002320210193F6F60F131837003B
:109B00001376F60F23261100232481001307F00F8C
:109B10009354F501138906001305060093D5F5014A
:109B2000939737006314E6006394070093C515000C
:109B30003387C640639A951A6356E00A6316060691
:109B4000639C07009307F00F638CF60493070800EB
:109B5000138506006F00C0141307F7FF631E07028A
:109B6000B38707011385060013975700635A07123E
:109B7000130515001307F00F630EE5323707007E5B
:109B800093F617001307F7FF93D71700B3F7E70013
:109B9000B3E7D7006F00C0101306F00F639EC60036
:109BA000930708006F0040071306F00FE38AC6FE14
:109BB00037060004B3E7C7001306B0016356E6009A
:109BC000930710006FF0DFF9130600023306E6403A
:109BD000B3D5E700B397C700B337F000B3E7F5009C
:109BE0006FF01FF863000708639C06026318080003
:109BF0001307F00F6316E60A6F0000029306F0FFEA
:109C00006316D700B38707016FF01FF69306F00FB6
:109C10001347F7FF6310D6021305F00F6F004008DB
:109C20009306F00FE30AD6FEB70600043307E040C0
:109C30003368D8009306B00163D6E600130710001E
:109C40006F00C001930600023356E8003387E640F8
:109C50003317E8003337E0003367E600B387E700E7
:109C60006FF09FF0138516001376F50F13071000A1
:109C70006342C706639406041305000063020802EA
:109C800063860722B387070113975700635A0700BB
:109C9000370700FC1307F7FFB3F7E70013051000C1
:109CA00013F77700630A072013F7F70093064000C5
:109CB0006304D720938747006F000020E30E08F469
:109CC000E38007EEB70700021305F00F93040000CE
:109CD0006F00801E1307F00F630EE51C3307F800BA
:109CE000935717006FF0DFFB6350E008631606041C
:109CF000E38A07E41307F7FF63140702B307F8408A
:109D00001385060013975700E35C07F83704000437
:109D10001304F4FF33F48700130905006F00801368
:109D20001306F00FE38EC6E61306B0016350E60299
:109D3000930710006FF09FFC1306F00FE382C6E656
:109D400037060004B3E7C7006FF01FFE13060002DA
:109D5000B3D5E7003307E640B397E700B337F00029
:109D6000B3E7F5006FF09FF963020708639E0602F0
:109D7000631808001307F00F938405006FF09FE746
:109D80009306F0FF6318D700B3870741938405005B
:109D90006FF05FF79306F00F1347F7FF6310D602DB
:109DA000938405006FF05FE79306F00FE30AD6FE99
:109DB000B70600043307E0403368D8009306B001CB
:109DC00063D6E600130710006F00C001930600027F
:109DD0003356E8003387E6403317E8003337E000B6
:109DE0003367E600B387E7406FF05FFA138716002A
:109DF0001377F70F130610006344E604639C060212
:109E00006318080063980712130500006FF01FEC39
:109E1000638607123307F84093165700B38707414C
:109E200063CA061093070700631007069307000034
:109E30006FF09FFDE31608E8E39407F66FF09FE8E4
:109E40003304F84013175400635407043384074164
:109E50009384050013050400EF00C01C1305B5FF33
:109E60003314A400634A2503330525411305150067
:109E700013070002B357A4003305A7403314A4000E
:109E800033348000B3E78700130500006FF05FE113
:109E9000E30E04F86FF01FFCB70700FC9387F7FF91
:109EA0003305A940B377F4006FF09FDF93070800F4
:109EB0006FF01FDF9307000013975700635E0700E2
:109EC000130515001307F00F630EE506370700FCB6
:109ED0001307F7FFB3F7E7001307F00F93D7370027
:109EE0006318E50063860700B7074000930400008D
:109EF000370780001307F7FF1375F50FB3F7E70077
:109F000013177501370580808320C1000324810069
:109F10001305F5FF33F5A7009394F4013365E500CD
:109F200033659500032901008324410013010101D9
:109F300067800000938405006FF01FF59307080009
:109F40006FF09FF4930700006FF01FF913060500F0
:109F50001305000093F61500638406003305C50061
:109F600093D5150013161600E39605FE67800000D2
:109F70006340050663C605061386050093050500C4
:109F80001305F0FF630C060293061000637AB60017
:109F90006358C0001316160093961600E36AB6FEC7
:109FA0001305000063E6C500B385C5403365D500E1
:109FB00093D6160013561600E39606FE678000003F
:109FC00093820000EFF05FFB1385050067800200BD
:109FD0003305A04063D80500B305B0406FF0DFF94A
:109FE000B305B04093820000EFF01FF93305A040A5
:109FF000678002009382000063CA0500634C05007D
:10A00000EFF09FF71385050067800200B305B040AD
:10A01000E35805FE3305A040EFF01FF63305B040CE
:10A0200067800200B7070100637AF5029307F00F1B
:10A03000B3B7A70093973700130700023307F74021
:10A04000B357F500176501001305452EB307F5005A
:10A0500003C507003305A7406780000037070001EC
:10A0600093070001E36AE5FC930780016FF0DFFCD2
:10A07000976701009387075983A6070017670100B8
:10A08000130707570327070023A2A600637EE500F6
:10A0900017670100130787560325070083A50700EC
:10A0A000938545006F600FEE130101FF23248100AB
:10A0B00023261100176701001307875413040500B6
:10A0C0000325070083A5070093854500EF608FEB0C
:10A0D000976701009387075083A707006376F40012
:10A0E0009767010023A8874E8320C10003248100C5
:10A0F0001301010167800000976701009387875073
:10A1000003A7070083A60700832747049387F7FF69
:10A110002322F70483A74604639407007360043086
:10A1200067800000130101FE232C8100232A910087
:10A1300013040500938405002328210123263101FF
:10A140002324410123225101232E1100EF80DF9FA0
:10A150008327040003290401B7090001B3E5970030
:10A16000930AC4002320B400930400009389F9FFEC
:10A17000370A00020327040063822A050326090028
:10A1800013050900B3654701B376360193175600EE
:10A1900033F7E6000329490063C60700631607008A
:10A1A0006FF05FFDE398E6FC9317760063D4070039
:10A1B000B3E4D400EF909FE16FF0DFFB93C4F4FFB2
:10A1C000B3F4E40023209400EF809FCB0325040028
:10A1D0008320C1010324810183244101032901015A
:10A1E0008329C100032A8100832A4100130101024F
:10A1F00067800000130101FF1305000023261100F2
:10A2000023248100EFD0DF8617D7FFFF1307C7D2C3
:10A210009306000013061000930540061765010021
:10A2200013058525EFB0CF906302050213040500E6
:10A23000EF801F931306050013070000930600002C
:10A240009305100013050400EFB08FA0EF800FDD21
:10A250008320C100032481001305000013010101C4
:04A260006780000013
:02000004800278
:100000004C63FEFFBC64FEFF5863FEFFBC64FEFF52
:10001000BC64FEFFBC64FEFFBC64FEFF8063FEFFA9
:10002000BC64FEFFBC64FEFFA863FEFFB863FEFF76
:10003000BC64FEFFD063FEFFE063FEFFE063FEFFF3
:10004000E063FEFFE063FEFFE063FEFFE063FEFFB0
:10005000E063FEFFE063FEFFE063FEFFBC64FEFFC3
:10006000BC64FEFFBC64FEFFBC64FEFFBC64FEFF1C
:10007000BC64FEFFBC64FEFFBC64FEFFBC64FEFF0C
:10008000BC64FEFFBC64FEFFBC64FEFFBC64FEFFFC
:10009000BC64FEFFBC64FEFFBC64FEFFBC64FEFFEC
:1000A000BC64FEFFBC64FEFFBC64FEFFBC64FEFFDC
:1000B000BC64FEFFBC64FEFFBC64FEFFBC64FEFFCC
:1000C000BC64FEFFBC64FEFFBC64FEFFBC64FEFFBC
:1000D000BC64FEFFBC64FEFFBC64FEFFBC64FEFFAC
:1000E000BC64FEFFBC64FEFFBC64FEFFBC64FEFF9C
:1000F000BC64FEFFBC64FEFFBC64FEFFBC64FEFF8C
:100100002464FEFF4C64FEFFBC64FEFFBC64FEFF83
:10011000BC64FEFFBC64FEFFBC64FEFFBC64FEFF6B
:10012000BC64FEFFAC64FEFFBC64FEFFBC64FEFF6B
:100130005C61FEFF6462FEFFBC64FEFFBC64FEFF08
:10014000B462FEFFBC64FEFF2C63FEFFBC64FEFFD6
:10015000BC64FEFF7463FEFF1869FEFF8469FEFF46
:100160002469FEFF8469FEFF8469FEFF8469FEFF47
:100170008469FEFFBC67FEFF8469FEFF8469FEFFA1
:10018000E467FEFFF467FEFF8469FEFF0C68FEFF74
:100190001C68FEFF1C68FEFF1C68FEFF1C68FEFF5B
:1001A0001C68FEFF1C68FEFF1C68FEFF1C68FEFF4B
:1001B0001C68FEFF8469FEFF8469FEFF8469FEFF00
:1001C0008469FEFF8469FEFF8469FEFF8469FEFF87
:1001D0008469FEFF8469FEFF8469FEFF8469FEFF77
:1001E0008469FEFF8469FEFF8469FEFF8469FEFF67
:1001F0008469FEFF8469FEFF8469FEFF8469FEFF57
:100200008469FEFF8469FEFF8469FEFF8469FEFF46
:100210008469FEFF8469FEFF8469FEFF8469FEFF36
:100220008469FEFF8469FEFF8469FEFF8469FEFF26
:100230008469FEFF8469FEFF8469FEFF8469FEFF16
:100240008469FEFF8469FEFF8469FEFF8469FEFF06
:100250008469FEFF8469FEFF6068FEFF9C68FEFF04
:100260008469FEFF8469FEFF8469FEFF8469FEFFE6
:100270008469FEFF8469FEFF8469FEFF0869FEFF52
:100280008469FEFF8469FEFF9065FEFFE466FEFF61
:100290008469FEFF8469FEFF7467FEFF8469FEFFC8
:1002A000A067FEFF8469FEFF8469FEFF7869FEFF98
:1002B0000092FEFF3C92FEFF4892FEFF3C92FEFF42
:1002C000B492FEFF3C92FEFF4892FEFF0092FEFFBA
:1002D0000092FEFFB492FEFF4892FEFF1892FEFFCE
:1002E0001892FEFF1892FEFF5092FEFFD896FEFF76
:1002F000D896FEFF5897FEFFD096FEFFD096FEFFE1
:10030000B897FEFF5897FEFFD096FEFFB897FEFF06
:10031000D096FEFF5897FEFFCC96FEFFCC96FEFFD0
:10032000CC96FEFFB897FEFF000102020303030311
:100330000404040404040404050505050505050575
:100340000505050505050505060606060606060655
:10035000060606060606060606060606060606063D
:100360000606060606060606070707070707070725
:10037000070707070707070707070707070707070D
:1003800007070707070707070707070707070707FD
:1003900007070707070707070707070707070707ED
:1003A00007070707070707070808080808080808D5
:1003B00008080808080808080808080808080808BD
:1003C00008080808080808080808080808080808AD
:1003D000080808080808080808080808080808089D
:1003E000080808080808080808080808080808088D
:1003F000080808080808080808080808080808087D
:10040000080808080808080808080808080808086C
:10041000080808080808080808080808080808085C
:100420000808080808080808546D72510000000008
:10043000546D722053766300286E756C6C29000031
:100440004572726F7220696E2073705F666C6F7098
:1004500073207461736B73200D0A00006D69616F06
:10046000750A00006D69616F75320A0068756E6704
:1004700072790A00436865636B54696D65720000A8
:100480004D617468310000004D61746832000000F5
:100490004D617468330000004D61746834000000E1
:1004A0004D617468350000004D61746836000000CD
:1004B0004D617468370000004D61746838000000B9
:1004C0001000000000000000017A5200017C0101D0
:1004D0001B0D02005000000018000000D078FEFF45
:1004E0005805000000440E507489039406990B814E
:1004F00001880292049305950796089709980A9A2D
:100500000C9B0D036C010AC144C844C944D244D3B6
:1005100044D444D544D644D744D844D944DA44DBFF
:10052000440E00440B0000004C0000006C00000072
:10053000D47DFEFFDC05000000440E307089039579
:1005400007810188029204930594069608970998FA
:100550000A990B9A0C0370020AC144C844C944D2D8
:1005600044D344D444D544D644D744D844D944DAB7
:10057000440E00440B00000050000000BC000000CE
:100580006083FEFF0005000000440E50748802895D
:10059000039305990B810192049406950796089799
:1005A00009980A9A0C9B0D0320010AC144C844C94A
:1005B00044D244D344D444D544D644D744D844D96F
:0C05C00044DA44DB440E00440B00000051
:10063400D5E9F642DD9A1245358E65C46F12833AC8
:10064400A4B0C2C366E4FD46A30100C0CFF7414194
:100654006F1283BA0000B040FC8F01000900000053
:040000058000004037
:00000001FF
